 getlocal001

 Timestamp is 0199e474 (reproducible build file hash)

 Preferred load address is 0000000180000000

 Start         Length     Name                   Class
 0001:00000000 00003b50H .text$mn                CODE
 0001:00003b50 00000036H .text$mn$00             CODE
 0001:00003b86 00000092H .text$x                 CODE
 0002:00000000 00000198H .idata$5                DATA
 0002:00000198 00000038H .00cfg                  DATA
 0002:000001d0 00000008H .CRT$XCA                DATA
 0002:000001d8 00000008H .CRT$XCZ                DATA
 0002:000001e0 00000008H .CRT$XIA                DATA
 0002:000001e8 00000008H .CRT$XIC                DATA
 0002:000001f0 00000008H .CRT$XIZ                DATA
 0002:000001f8 00000008H .CRT$XLA                DATA
 0002:00000200 00000008H .CRT$XLZ                DATA
 0002:00000208 00000008H .CRT$XPA                DATA
 0002:00000210 00000008H .CRT$XPZ                DATA
 0002:00000218 00000008H .CRT$XTA                DATA
 0002:00000220 00000010H .CRT$XTZ                DATA
 0002:00000228 00000000H .gehcont$y              DATA
 0002:00000228 00000000H .gfids$y                DATA
 0002:00000230 000023d0H .rdata                  DATA
 0002:00002600 00000000H .rdata$CastGuardVftablesA DATA
 0002:00002600 00000000H .rdata$CastGuardVftablesC DATA
 0002:00002600 00000028H .rdata$T                DATA
 0002:00002628 000000b0H .rdata$voltmd           DATA
 0002:000026d8 00000318H .rdata$zzzdbg           DATA
 0002:000029f0 00000008H .rtc$IAA                DATA
 0002:000029f8 00000008H .rtc$IZZ                DATA
 0002:00002a00 00000008H .rtc$TAA                DATA
 0002:00002a08 00000008H .rtc$TZZ                DATA
 0002:00002a10 00000004H .tls                    DATA
 0002:00002a14 00000004H .tls$                   DATA
 0002:00002a18 00000008H .tls$ZZZ                DATA
 0002:00002a20 00000380H .xdata                  DATA
 0002:00002da0 000003e0H .edata                  DATA
 0002:00003180 00000064H .idata$2                DATA
 0002:000031e4 00000014H .idata$3                DATA
 0002:000031f8 00000198H .idata$4                DATA
 0002:00003390 0000041eH .idata$6                DATA
 0003:00000000 00000080H .data                   DATA
 0003:00000080 0001b3a8H .bss                    DATA
 0004:00000000 000003b4H .pdata                  DATA

  Address         Publics by Value              Rva+Base               Lib:Object

 0000:00000000       __AbsoluteZero             0000000000000000     <absolute>
 0000:00000000       ___safe_se_handler_count   0000000000000000     <absolute>
 0000:00000000       ___safe_se_handler_table   0000000000000000     <absolute>
 0000:00000000       __arm64x_extra_rfe_table   0000000000000000     <absolute>
 0000:00000000       __arm64x_extra_rfe_table_size 0000000000000000     <absolute>
 0000:00000000       __arm64x_native_entrypoint 0000000000000000     <absolute>
 0000:00000000       __arm64x_redirection_metadata 0000000000000000     <absolute>
 0000:00000000       __arm64x_redirection_metadata_count 0000000000000000     <absolute>
 0000:00000000       __dynamic_value_reloc_table 0000000000000000     <absolute>
 0000:00000000       __enclave_config           0000000000000000     <absolute>
 0000:00000000       __guard_check_icall_a64n_fptr 0000000000000000     <absolute>
 0000:00000000       __guard_eh_cont_count      0000000000000000     <absolute>
 0000:00000000       __guard_eh_cont_table      0000000000000000     <absolute>
 0000:00000000       __guard_fids_count         0000000000000000     <absolute>
 0000:00000000       __guard_fids_table         0000000000000000     <absolute>
 0000:00000000       __guard_iat_count          0000000000000000     <absolute>
 0000:00000000       __guard_iat_table          0000000000000000     <absolute>
 0000:00000000       __guard_longjmp_count      0000000000000000     <absolute>
 0000:00000000       __guard_longjmp_table      0000000000000000     <absolute>
 0000:00000000       __hybrid_auxiliary_iat     0000000000000000     <absolute>
 0000:00000000       __hybrid_auxiliary_iat_copy 0000000000000000     <absolute>
 0000:00000000       __hybrid_code_map          0000000000000000     <absolute>
 0000:00000000       __hybrid_code_map_count    0000000000000000     <absolute>
 0000:00000000       __x64_code_ranges_to_entry_points 0000000000000000     <absolute>
 0000:00000000       __x64_code_ranges_to_entry_points_count 0000000000000000     <absolute>
 0000:00000100       __guard_flags              0000000000000100     <absolute>
 0000:00000000       __ImageBase                0000000180000000     <linker-defined>
 0001:00000000       ?NewObject@JNIEnv_@@QEAAPEAV_jobject@@PEAV_jclass@@PEAU_jmethodID@@ZZ 0000000180001000 f i libgetlocal001.obj
 0001:00000024       ?SetEventNotificationMode@_jvmtiEnv@@QEAA?AW4jvmtiError@@W4jvmtiEventMode@@W4jvmtiEvent@@PEAV_jobject@@ZZ 0000000180001024 f i libgetlocal001.obj
 0001:0000002c       ?TranslateError@@YAPEBDW4jvmtiError@@@Z 000000018000102c f   libgetlocal001.obj
 0001:000002e4       ?nsk_jni_check_exception@@YAHPEAUJNIEnv_@@QEBDH@Z 00000001800012e4 f   libgetlocal001.obj
 0001:00000428       ?nsk_jni_lverify@@YAHHPEAUJNIEnv_@@HQEBDH1ZZ 0000000180001428 f   libgetlocal001.obj
 0001:000004c8       Agent_Initialize           00000001800014c8 f   libgetlocal001.obj
 0001:00000654       Agent_OnAttach             0000000180001654 f   libgetlocal001.obj
 0001:00000654       Agent_OnLoad               0000000180001654 f   libgetlocal001.obj
 0001:0000065c       Breakpoint                 000000018000165c f   libgetlocal001.obj
 0001:00000888       Java_nsk_jvmti_GetLocalVariable_getlocal001_getMeth 0000000180001888 f   libgetlocal001.obj
 0001:00000aa0       Java_nsk_jvmti_GetLocalVariable_getlocal001_getRes 0000000180001aa0 f   libgetlocal001.obj
 0001:00000aa8       Java_nsk_jvmti_unit_FollowReferences_FollowRefObjects_addRefToVerify 0000000180001aa8 f   libgetlocal001.obj
 0001:00000c64       Java_nsk_jvmti_unit_FollowReferences_FollowRefObjects_getTag 0000000180001c64 f   libgetlocal001.obj
 0001:00000d20       Java_nsk_jvmti_unit_FollowReferences_FollowRefObjects_resetRefsToVerify 0000000180001d20 f   libgetlocal001.obj
 0001:00000d28       Java_nsk_jvmti_unit_FollowReferences_FollowRefObjects_resetTags 0000000180001d28 f   libgetlocal001.obj
 0001:00000d6c       Java_nsk_jvmti_unit_FollowReferences_FollowRefObjects_setTag 0000000180001d6c f   libgetlocal001.obj
 0001:00000fb8       Java_nsk_share_jvmti_ArgumentHandler_getAgentOptionsString 0000000180001fb8 f   libgetlocal001.obj
 0001:00001064       Java_nsk_share_jvmti_DebugeeClass_checkStatus 0000000180002064 f   libgetlocal001.obj
 0001:000010ec       Java_nsk_share_jvmti_DebugeeClass_resetAgentData 00000001800020ec f   libgetlocal001.obj
 0001:0000114c       Java_nsk_share_jvmti_RedefineAgent_agentStatus 000000018000214c f   libgetlocal001.obj
 0001:00001158       Java_nsk_share_jvmti_RedefineAgent_isRedefined 0000000180002158 f   libgetlocal001.obj
 0001:00001164       Java_nsk_share_jvmti_RedefineAgent_redefineAttempted 0000000180002164 f   libgetlocal001.obj
 0001:00001170       MA_checkStatus             0000000180002170 f   libgetlocal001.obj
 0001:00001214       MethodExit                 0000000180002214 f   libgetlocal001.obj
 0001:00001414       __local_stdio_printf_options 0000000180002414 f i libgetlocal001.obj
 0001:000015e4       check1                     00000001800025e4 f   libgetlocal001.obj
 0001:000017f0       check2                     00000001800027f0 f   libgetlocal001.obj
 0001:00001a78       check3                     0000000180002a78 f   libgetlocal001.obj
 0001:00001cb4       check4                     0000000180002cb4 f   libgetlocal001.obj
 0001:000020d4       exitOnError                00000001800030d4 f   libgetlocal001.obj
 0001:00002188       fprintf                    0000000180003188 f i libgetlocal001.obj
 0001:000021cc       nsk_jvmti_lverify          00000001800031cc f   libgetlocal001.obj
 0001:000022bc       nsk_jvmti_resetAgentData   00000001800032bc f   libgetlocal001.obj
 0001:00002330       nsk_lcomplain              0000000180003330 f   libgetlocal001.obj
 0001:00002350       nsk_ldisplay               0000000180003350 f   libgetlocal001.obj
 0001:00002370       nsk_ltrace                 0000000180003370 f   libgetlocal001.obj
 0001:00002390       nsk_lvcomplain             0000000180003390 f   libgetlocal001.obj
 0001:00002548       nsk_lvdisplay              0000000180003548 f   libgetlocal001.obj
 0001:00002594       nsk_lverify                0000000180003594 f   libgetlocal001.obj
 0001:000025f0       nsk_lvtrace                00000001800035f0 f   libgetlocal001.obj
 0001:00002650       nsk_printf                 0000000180003650 f   libgetlocal001.obj
 0001:00002678       nsk_vprintf                0000000180003678 f   libgetlocal001.obj
 0001:0000272c       printf                     000000018000372c f i libgetlocal001.obj
 0001:00002c2c       __raise_securityfailure    0000000180003c2c f   MSVCRT:gs_report.obj
 0001:00002c60       __report_gsfailure         0000000180003c60 f   MSVCRT:gs_report.obj
 0001:00002ea0       __GSHandlerCheck           0000000180003ea0 f   MSVCRT:gshandler.obj
 0001:00002ec0       __GSHandlerCheckCommon     0000000180003ec0 f   MSVCRT:gshandler.obj
 0001:00002f30       __security_check_cookie    0000000180003f30 f   MSVCRT:amdsecgs.obj
 0001:00003270       _DllMainCRTStartup         0000000180004270 f   MSVCRT:dll_dllmain.obj
 0001:000032b0       __scrt_acquire_startup_lock 00000001800042b0 f   MSVCRT:utility.obj
 0001:000032ec       __scrt_dllmain_after_initialize_c 00000001800042ec f   MSVCRT:utility.obj
 0001:00003320       __scrt_dllmain_before_initialize_c 0000000180004320 f   MSVCRT:utility.obj
 0001:00003338       __scrt_dllmain_crt_thread_attach 0000000180004338 f   MSVCRT:utility.obj
 0001:00003360       __scrt_dllmain_crt_thread_detach 0000000180004360 f   MSVCRT:utility.obj
 0001:00003378       __scrt_dllmain_exception_filter 0000000180004378 f   MSVCRT:utility.obj
 0001:000033d8       __scrt_dllmain_uninitialize_c 00000001800043d8 f   MSVCRT:utility.obj
 0001:00003408       __scrt_dllmain_uninitialize_critical 0000000180004408 f   MSVCRT:utility.obj
 0001:0000341c       __scrt_initialize_crt      000000018000441c f   MSVCRT:utility.obj
 0001:00003468       __scrt_initialize_onexit_tables 0000000180004468 f   MSVCRT:utility.obj
 0001:000034f4       __scrt_is_nonwritable_in_current_image 00000001800044f4 f   MSVCRT:utility.obj
 0001:0000358c       __scrt_release_startup_lock 000000018000458c f   MSVCRT:utility.obj
 0001:000035b0       __scrt_uninitialize_crt    00000001800045b0 f   MSVCRT:utility.obj
 0001:000035dc       _onexit                    00000001800045dc f   MSVCRT:utility.obj
 0001:00003618       atexit                     0000000180004618 f   MSVCRT:utility.obj
 0001:00003630       __crt_debugger_hook        0000000180004630 f   MSVCRT:utility_desktop.obj
 0001:00003638       __scrt_fastfail            0000000180004638 f   MSVCRT:utility_desktop.obj
 0001:00003784       _guard_check_icall_nop     0000000180004784 f i MSVCRT:guard_support.obj
 0001:00003788       __security_init_cookie     0000000180004788 f   MSVCRT:gs_support.obj
 0001:00003834       DllMain                    0000000180004834 f   MSVCRT:dll_dllmain_stub.obj
 0001:00003858       ?__scrt_initialize_type_info@@YAXXZ 0000000180004858 f   MSVCRT:tncleanup.obj
 0001:00003868       ?__scrt_uninitialize_type_info@@YAXXZ 0000000180004868 f   MSVCRT:tncleanup.obj
 0001:00003874       __local_stdio_scanf_options 0000000180004874 f i MSVCRT:default_local_stdio_options.obj
 0001:0000387c       __scrt_initialize_default_local_stdio_options 000000018000487c f   MSVCRT:default_local_stdio_options.obj
 0001:00003898       __scrt_get_dyn_tls_init_callback 0000000180004898 f   MSVCRT:dyn_tls_init.obj
 0001:000038a0       _RTC_Initialize            00000001800048a0 f   MSVCRT:initsect.obj
 0001:000038dc       _RTC_Terminate             00000001800048dc f   MSVCRT:initsect.obj
 0001:00003918       __isa_available_init       0000000180004918 f   MSVCRT:cpu_disp.obj
 0001:00003ac4       _get_startup_argv_mode     0000000180004ac4 f   MSVCRT:argv_mode.obj
 0001:00003acc       __scrt_is_ucrt_dll_in_use  0000000180004acc f   MSVCRT:ucrt_detection.obj
 0001:00003ae0       memcpy                     0000000180004ae0 f   vcruntime:VCRUNTIME140.dll
 0001:00003ae6       memset                     0000000180004ae6 f   vcruntime:VCRUNTIME140.dll
 0001:00003aec       strchr                     0000000180004aec f   vcruntime:VCRUNTIME140.dll
 0001:00003af2       __C_specific_handler       0000000180004af2 f   vcruntime:VCRUNTIME140.dll
 0001:00003af8       __std_type_info_destroy_list 0000000180004af8 f   vcruntime:VCRUNTIME140.dll
 0001:00003afe       strcmp                     0000000180004afe f   ucrt:api-ms-win-crt-string-l1-1-0.dll
 0001:00003b04       strlen                     0000000180004b04 f   ucrt:api-ms-win-crt-string-l1-1-0.dll
 0001:00003b0a       _initterm                  0000000180004b0a f   ucrt:api-ms-win-crt-runtime-l1-1-0.dll
 0001:00003b10       _initterm_e                0000000180004b10 f   ucrt:api-ms-win-crt-runtime-l1-1-0.dll
 0001:00003b16       _seh_filter_dll            0000000180004b16 f   ucrt:api-ms-win-crt-runtime-l1-1-0.dll
 0001:00003b1c       _configure_narrow_argv     0000000180004b1c f   ucrt:api-ms-win-crt-runtime-l1-1-0.dll
 0001:00003b22       _initialize_narrow_environment 0000000180004b22 f   ucrt:api-ms-win-crt-runtime-l1-1-0.dll
 0001:00003b28       _initialize_onexit_table   0000000180004b28 f   ucrt:api-ms-win-crt-runtime-l1-1-0.dll
 0001:00003b2e       _register_onexit_function  0000000180004b2e f   ucrt:api-ms-win-crt-runtime-l1-1-0.dll
 0001:00003b34       _execute_onexit_table      0000000180004b34 f   ucrt:api-ms-win-crt-runtime-l1-1-0.dll
 0001:00003b3a       _crt_atexit                0000000180004b3a f   ucrt:api-ms-win-crt-runtime-l1-1-0.dll
 0001:00003b40       _cexit                     0000000180004b40 f   ucrt:api-ms-win-crt-runtime-l1-1-0.dll
 0001:00003b48       __acrt_initialize          0000000180004b48 f   MSVCRT:ucrt_stubs.obj
 0001:00003b48       __acrt_thread_attach       0000000180004b48 f   MSVCRT:ucrt_stubs.obj
 0001:00003b48       __acrt_thread_detach       0000000180004b48 f   MSVCRT:ucrt_stubs.obj
 0001:00003b48       __acrt_uninitialize        0000000180004b48 f   MSVCRT:ucrt_stubs.obj
 0001:00003b48       __acrt_uninitialize_critical 0000000180004b48 f   MSVCRT:ucrt_stubs.obj
 0001:00003b48       __scrt_stub_for_acrt_initialize 0000000180004b48 f   MSVCRT:ucrt_stubs.obj
 0001:00003b48       __scrt_stub_for_acrt_thread_attach 0000000180004b48 f   MSVCRT:ucrt_stubs.obj
 0001:00003b48       __scrt_stub_for_acrt_thread_detach 0000000180004b48 f   MSVCRT:ucrt_stubs.obj
 0001:00003b48       __scrt_stub_for_acrt_uninitialize 0000000180004b48 f   MSVCRT:ucrt_stubs.obj
 0001:00003b48       __scrt_stub_for_acrt_uninitialize_critical 0000000180004b48 f   MSVCRT:ucrt_stubs.obj
 0001:00003b48       __vcrt_initialize          0000000180004b48 f   MSVCRT:ucrt_stubs.obj
 0001:00003b48       __vcrt_thread_attach       0000000180004b48 f   MSVCRT:ucrt_stubs.obj
 0001:00003b48       __vcrt_thread_detach       0000000180004b48 f   MSVCRT:ucrt_stubs.obj
 0001:00003b48       __vcrt_uninitialize        0000000180004b48 f   MSVCRT:ucrt_stubs.obj
 0001:00003b48       __vcrt_uninitialize_critical 0000000180004b48 f   MSVCRT:ucrt_stubs.obj
 0001:00003b4c       __scrt_stub_for_is_c_termination_complete 0000000180004b4c f   MSVCRT:ucrt_stubs.obj
 0001:00003b4c       _is_c_termination_complete 0000000180004b4c f   MSVCRT:ucrt_stubs.obj
 0001:00003b60       _guard_dispatch_icall_nop  0000000180004b60 f   MSVCRT:guard_dispatch.obj
 0001:00003b80       _guard_xfg_dispatch_icall_nop 0000000180004b80 f   MSVCRT:guard_xfg_dispatch.obj
 0002:00000000       __imp_RtlCaptureContext    0000000180005000     kernel32:KERNEL32.dll
 0002:00000008       __imp_RtlLookupFunctionEntry 0000000180005008     kernel32:KERNEL32.dll
 0002:00000010       __imp_RtlVirtualUnwind     0000000180005010     kernel32:KERNEL32.dll
 0002:00000018       __imp_UnhandledExceptionFilter 0000000180005018     kernel32:KERNEL32.dll
 0002:00000020       __imp_SetUnhandledExceptionFilter 0000000180005020     kernel32:KERNEL32.dll
 0002:00000028       __imp_GetCurrentProcess    0000000180005028     kernel32:KERNEL32.dll
 0002:00000030       __imp_TerminateProcess     0000000180005030     kernel32:KERNEL32.dll
 0002:00000038       __imp_IsProcessorFeaturePresent 0000000180005038     kernel32:KERNEL32.dll
 0002:00000040       __imp_CloseHandle          0000000180005040     kernel32:KERNEL32.dll
 0002:00000048       __imp_InitializeCriticalSectionAndSpinCount 0000000180005048     kernel32:KERNEL32.dll
 0002:00000050       __imp_DeleteCriticalSection 0000000180005050     kernel32:KERNEL32.dll
 0002:00000058       __imp_CreateEventW         0000000180005058     kernel32:KERNEL32.dll
 0002:00000060       __imp_GetModuleHandleW     0000000180005060     kernel32:KERNEL32.dll
 0002:00000068       __imp_GetProcAddress       0000000180005068     kernel32:KERNEL32.dll
 0002:00000070       __imp_IsDebuggerPresent    0000000180005070     kernel32:KERNEL32.dll
 0002:00000078       __imp_QueryPerformanceCounter 0000000180005078     kernel32:KERNEL32.dll
 0002:00000080       __imp_GetCurrentProcessId  0000000180005080     kernel32:KERNEL32.dll
 0002:00000088       __imp_GetCurrentThreadId   0000000180005088     kernel32:KERNEL32.dll
 0002:00000090       __imp_GetSystemTimeAsFileTime 0000000180005090     kernel32:KERNEL32.dll
 0002:00000098       __imp_DisableThreadLibraryCalls 0000000180005098     kernel32:KERNEL32.dll
 0002:000000a0       __imp_InitializeSListHead  00000001800050a0     kernel32:KERNEL32.dll
 0002:000000a8       \177KERNEL32_NULL_THUNK_DATA 00000001800050a8     kernel32:KERNEL32.dll
 0002:000000b0       __imp_memcpy               00000001800050b0     vcruntime:VCRUNTIME140.dll
 0002:000000b8       __imp_memset               00000001800050b8     vcruntime:VCRUNTIME140.dll
 0002:000000c0       __imp_strchr               00000001800050c0     vcruntime:VCRUNTIME140.dll
 0002:000000c8       __imp___C_specific_handler 00000001800050c8     vcruntime:VCRUNTIME140.dll
 0002:000000d0       __imp___std_type_info_destroy_list 00000001800050d0     vcruntime:VCRUNTIME140.dll
 0002:000000d8       \177VCRUNTIME140_NULL_THUNK_DATA 00000001800050d8     vcruntime:VCRUNTIME140.dll
 0002:000000e0       __imp__errno               00000001800050e0     ucrt:api-ms-win-crt-runtime-l1-1-0.dll
 0002:000000e8       __imp_exit                 00000001800050e8     ucrt:api-ms-win-crt-runtime-l1-1-0.dll
 0002:000000f0       __imp__cexit               00000001800050f0     ucrt:api-ms-win-crt-runtime-l1-1-0.dll
 0002:000000f8       __imp__crt_atexit          00000001800050f8     ucrt:api-ms-win-crt-runtime-l1-1-0.dll
 0002:00000100       __imp__execute_onexit_table 0000000180005100     ucrt:api-ms-win-crt-runtime-l1-1-0.dll
 0002:00000108       __imp__register_onexit_function 0000000180005108     ucrt:api-ms-win-crt-runtime-l1-1-0.dll
 0002:00000110       __imp__initialize_onexit_table 0000000180005110     ucrt:api-ms-win-crt-runtime-l1-1-0.dll
 0002:00000118       __imp__initialize_narrow_environment 0000000180005118     ucrt:api-ms-win-crt-runtime-l1-1-0.dll
 0002:00000120       __imp__configure_narrow_argv 0000000180005120     ucrt:api-ms-win-crt-runtime-l1-1-0.dll
 0002:00000128       __imp__seh_filter_dll      0000000180005128     ucrt:api-ms-win-crt-runtime-l1-1-0.dll
 0002:00000130       __imp__initterm_e          0000000180005130     ucrt:api-ms-win-crt-runtime-l1-1-0.dll
 0002:00000138       __imp__initterm            0000000180005138     ucrt:api-ms-win-crt-runtime-l1-1-0.dll
 0002:00000140       \177api-ms-win-crt-runtime-l1-1-0_NULL_THUNK_DATA 0000000180005140     ucrt:api-ms-win-crt-runtime-l1-1-0.dll
 0002:00000148       __imp___acrt_iob_func      0000000180005148     ucrt:api-ms-win-crt-stdio-l1-1-0.dll
 0002:00000150       __imp_fflush               0000000180005150     ucrt:api-ms-win-crt-stdio-l1-1-0.dll
 0002:00000158       __imp___stdio_common_vsprintf 0000000180005158     ucrt:api-ms-win-crt-stdio-l1-1-0.dll
 0002:00000160       __imp___stdio_common_vfprintf 0000000180005160     ucrt:api-ms-win-crt-stdio-l1-1-0.dll
 0002:00000168       \177api-ms-win-crt-stdio-l1-1-0_NULL_THUNK_DATA 0000000180005168     ucrt:api-ms-win-crt-stdio-l1-1-0.dll
 0002:00000170       __imp_strcmp               0000000180005170     ucrt:api-ms-win-crt-string-l1-1-0.dll
 0002:00000178       __imp__strdup              0000000180005178     ucrt:api-ms-win-crt-string-l1-1-0.dll
 0002:00000178       __imp_strdup               0000000180005178     ucrt:api-ms-win-crt-string-l1-1-0.dll
 0002:00000180       __imp_strlen               0000000180005180     ucrt:api-ms-win-crt-string-l1-1-0.dll
 0002:00000188       __imp_strncpy              0000000180005188     ucrt:api-ms-win-crt-string-l1-1-0.dll
 0002:00000190       \177api-ms-win-crt-string-l1-1-0_NULL_THUNK_DATA 0000000180005190     ucrt:api-ms-win-crt-string-l1-1-0.dll
 0002:00000198       __guard_check_icall_fptr   0000000180005198     MSVCRT:guard_support.obj
 0002:000001a0       __guard_xfg_check_icall_fptr 00000001800051a0     MSVCRT:guard_support.obj
 0002:000001a8       __guard_dispatch_icall_fptr 00000001800051a8     MSVCRT:guard_support.obj
 0002:000001b0       __guard_xfg_dispatch_icall_fptr 00000001800051b0     MSVCRT:guard_support.obj
 0002:000001b8       __guard_xfg_table_dispatch_icall_fptr 00000001800051b8     MSVCRT:guard_support.obj
 0002:000001c0       __castguard_check_failure_os_handled_fptr 00000001800051c0     MSVCRT:guard_support.obj
 0002:000001c8       __guard_memcpy_fptr        00000001800051c8     vcruntime:softmemtag.obj
 0002:000001d0       __xc_a                     00000001800051d0     MSVCRT:initializers.obj
 0002:000001d8       __xc_z                     00000001800051d8     MSVCRT:initializers.obj
 0002:000001e0       __xi_a                     00000001800051e0     MSVCRT:initializers.obj
 0002:000001f0       __xi_z                     00000001800051f0     MSVCRT:initializers.obj
 0002:000001f8       __xl_a                     00000001800051f8     MSVCRT:tlssup.obj
 0002:00000200       __xl_z                     0000000180005200     MSVCRT:tlssup.obj
 0002:00000208       __xp_a                     0000000180005208     MSVCRT:initializers.obj
 0002:00000210       __xp_z                     0000000180005210     MSVCRT:initializers.obj
 0002:00000218       __xt_a                     0000000180005218     MSVCRT:initializers.obj
 0002:00000220       __xt_z                     0000000180005220     MSVCRT:initializers.obj
 0002:00000230       g_refKindStr               0000000180005230     libgetlocal001.obj
 0002:000003e0       ??_C@_09BPLDFGCI@unknown_0@ 00000001800053e0     libgetlocal001.obj
 0002:000003f0       ??_C@_0BL@FPNMECJD@JVMTI_HEAP_REFERENCE_CLASS@ 00000001800053f0     libgetlocal001.obj
 0002:00000410       ??_C@_0BL@FKGKKLNM@JVMTI_HEAP_REFERENCE_FIELD@ 0000000180005410     libgetlocal001.obj
 0002:00000430       ??_C@_0CD@CAEHCFJF@JVMTI_HEAP_REFERENCE_ARRAY_ELEM@ 0000000180005430     libgetlocal001.obj
 0002:00000458       ??_C@_0CC@DNEBMCNK@JVMTI_HEAP_REFERENCE_CLASS_LOAD@ 0000000180005458     libgetlocal001.obj
 0002:00000480       ??_C@_0BN@CJMIPEBB@JVMTI_HEAP_REFERENCE_SIGNERS@ 0000000180005480     libgetlocal001.obj
 0002:000004a0       ??_C@_0CH@HBOIDPEB@JVMTI_HEAP_REFERENCE_PROTECTION@ 00000001800054a0     libgetlocal001.obj
 0002:000004c8       ??_C@_0BP@MDKGDGKL@JVMTI_HEAP_REFERENCE_INTERFACE@ 00000001800054c8     libgetlocal001.obj
 0002:000004e8       ??_C@_0CC@JJMIHNJH@JVMTI_HEAP_REFERENCE_STATIC_FIE@ 00000001800054e8     libgetlocal001.obj
 0002:00000510       ??_C@_0CD@IDHEEGID@JVMTI_HEAP_REFERENCE_CONSTANT_P@ 0000000180005510     libgetlocal001.obj
 0002:00000538       ??_C@_0CA@EFFCHNG@JVMTI_HEAP_REFERENCE_SUPERCLASS@ 0000000180005538     libgetlocal001.obj
 0002:00000558       ??_C@_0L@PCDFHGCJ@unknown_11@ 0000000180005558     libgetlocal001.obj
 0002:00000568       ??_C@_0L@NJBICFOK@unknown_12@ 0000000180005568     libgetlocal001.obj
 0002:00000578       ??_C@_0L@MAADBEKL@unknown_13@ 0000000180005578     libgetlocal001.obj
 0002:00000588       ??_C@_0L@IPECICGM@unknown_14@ 0000000180005588     libgetlocal001.obj
 0002:00000598       ??_C@_0L@JGFJLDCN@unknown_15@ 0000000180005598     libgetlocal001.obj
 0002:000005a8       ??_C@_0L@LNHEOAOO@unknown_16@ 00000001800055a8     libgetlocal001.obj
 0002:000005b8       ??_C@_0L@KEGPNBKP@unknown_17@ 00000001800055b8     libgetlocal001.obj
 0002:000005c8       ??_C@_0L@CDPHMNGA@unknown_18@ 00000001800055c8     libgetlocal001.obj
 0002:000005d8       ??_C@_0L@DKOMPMCB@unknown_19@ 00000001800055d8     libgetlocal001.obj
 0002:000005e8       ??_C@_0L@OJGIPJDB@unknown_20@ 00000001800055e8     libgetlocal001.obj
 0002:000005f8       ??_C@_0CA@KAOFNDEM@JVMTI_HEAP_REFERENCE_JNI_GLOBAL@ 00000001800055f8     libgetlocal001.obj
 0002:00000618       ??_C@_0CC@HPFAJBK@JVMTI_HEAP_REFERENCE_SYSTEM_CLA@ 0000000180005618     libgetlocal001.obj
 0002:00000640       ??_C@_0BN@FDEGFOHC@JVMTI_HEAP_REFERENCE_MONITOR@ 0000000180005640     libgetlocal001.obj
 0002:00000660       ??_C@_0CB@HKIBCMAJ@JVMTI_HEAP_REFERENCE_STACK_LOCA@ 0000000180005660     libgetlocal001.obj
 0002:00000688       ??_C@_0BP@EAACMMOE@JVMTI_HEAP_REFERENCE_JNI_LOCAL@ 0000000180005688     libgetlocal001.obj
 0002:000006a8       ??_C@_0BM@IJDEOGOE@JVMTI_HEAP_REFERENCE_THREAD@ 00000001800056a8     libgetlocal001.obj
 0002:000006c8       ??_C@_0BL@EDGPPKC@JVMTI_HEAP_REFERENCE_OTHER@ 00000001800056c8     libgetlocal001.obj
 0002:000006e4       ??_C@_04BCJPDBDA@Code@     00000001800056e4     libgetlocal001.obj
 0002:000006f0       ??_C@_0BA@OCLMCFKC@LineNumberTable@ 00000001800056f0     libgetlocal001.obj
 0002:00000700       ??_C@_0BD@CPAEPILC@LocalVariableTable@ 0000000180005700     libgetlocal001.obj
 0002:00000718       ??_C@_0BH@NMBDNHBD@LocalVariableTypeTable@ 0000000180005718     libgetlocal001.obj
 0002:00000730       ??_C@_0O@HIHEEDNJ@StackMapTable@ 0000000180005730     libgetlocal001.obj
 0002:00000740       ??_C@_0L@HCDIAMJG@?9?5?$CFs?0?5?$CFd?3?5@ 0000000180005740     libgetlocal001.obj
 0002:00000750       ??_C@_0JI@HLPECLFI@?$CD?5?4?4?4?6?$CD?5ERROR?3?5too?5many?5complai@ 0000000180005750     libgetlocal001.obj
 0002:000007f0       ??_C@_0ED@JNEKCCOB@The?5following?5fake?5exception?5st@ 00000001800057f0     libgetlocal001.obj
 0002:00000838       ??_C@_0CN@FCNMDFBH@nsk?4share?4Fake_Exception_for_RU@ 0000000180005838     libgetlocal001.obj
 0002:00000868       ??_C@_08PGFFNAEI@?$CI?$CFs?3?$CFd?$CJ?5@ 0000000180005868     libgetlocal001.obj
 0002:00000878       ??_C@_0DP@IENMAEGI@s?2test?2hotspot?2jtreg?2vmTestbase@ 0000000180005878     libgetlocal001.obj
 0002:000008b8       ??_C@_0BL@NDJLFFJB@?7at?5nsk_lvcomplain?$CI?$CFs?3?$CFd?$CJ?6@ 00000001800058b8     libgetlocal001.obj
 0002:000008d8       ??_C@_0BC@JOOKAFKF@?$CD?5ERROR?3?5?$CFs?0?5?$CFd?3?5@ 00000001800058d8     libgetlocal001.obj
 0002:000008f0       ??_C@_09KJEAHMEH@?$CD?5ERROR?3?5@ 00000001800058f0     libgetlocal001.obj
 0002:000008fc       ??_C@_02GPIOPFAK@?$DO?$DO@ 00000001800058fc     libgetlocal001.obj
 0002:00000900       ??_C@_02FODMEDOG@?$DM?$DM@ 0000000180005900     libgetlocal001.obj
 0002:00000904       ??_C@_02DJGKEECL@?4?4@     0000000180005904     libgetlocal001.obj
 0002:00000908       ??_C@_0O@CJPGJOAF@?9?5?$CFs?0?5?$CFd?3?5?$CFs?5@ 0000000180005908     libgetlocal001.obj
 0002:00000918       ??_C@_0CB@IAKPDOIC@?$CD?5?5?5verified?5assertion?5is?5FALSE@ 0000000180005918     libgetlocal001.obj
 0002:00000940       ??_C@_0CO@LGONDEPD@stdout?3?5fflush?5failed?5?9?5err?$DN?$CFd?5@ 0000000180005940     libgetlocal001.obj
 0002:00000970       ??_C@_0CO@KBGKJPBD@stderr?3?5fflush?5failed?5?9?5err?$DN?$CFd?5@ 0000000180005970     libgetlocal001.obj
 0002:000009a0       ??_C@_0BB@JCNMKLLK@JVMTI_ERROR_NONE@ 00000001800059a0     libgetlocal001.obj
 0002:000009b8       ??_C@_0BL@LDIMKLPH@JVMTI_ERROR_INVALID_THREAD@ 00000001800059b8     libgetlocal001.obj
 0002:000009d8       ??_C@_0CB@PJFPAIKJ@JVMTI_ERROR_INVALID_THREAD_GROU@ 00000001800059d8     libgetlocal001.obj
 0002:00000a00       ??_C@_0BN@LLMKHMNF@JVMTI_ERROR_INVALID_PRIORITY@ 0000000180005a00     libgetlocal001.obj
 0002:00000a20       ??_C@_0CB@MBOFKAGB@JVMTI_ERROR_THREAD_NOT_SUSPENDE@ 0000000180005a20     libgetlocal001.obj
 0002:00000a48       ??_C@_0BN@FABOLPBI@JVMTI_ERROR_THREAD_SUSPENDED@ 0000000180005a48     libgetlocal001.obj
 0002:00000a68       ??_C@_0BN@FDGNOBJM@JVMTI_ERROR_THREAD_NOT_ALIVE@ 0000000180005a68     libgetlocal001.obj
 0002:00000a88       ??_C@_0BL@GOBIFKNJ@JVMTI_ERROR_INVALID_OBJECT@ 0000000180005a88     libgetlocal001.obj
 0002:00000aa8       ??_C@_0BK@FCMAJPPC@JVMTI_ERROR_INVALID_CLASS@ 0000000180005aa8     libgetlocal001.obj
 0002:00000ac8       ??_C@_0BP@IKLLBKEB@JVMTI_ERROR_CLASS_NOT_PREPARED@ 0000000180005ac8     libgetlocal001.obj
 0002:00000ae8       ??_C@_0BN@KLPPLKG@JVMTI_ERROR_INVALID_METHODID@ 0000000180005ae8     libgetlocal001.obj
 0002:00000b08       ??_C@_0BN@BCEKOKND@JVMTI_ERROR_INVALID_LOCATION@ 0000000180005b08     libgetlocal001.obj
 0002:00000b28       ??_C@_0BM@DFDGPME@JVMTI_ERROR_INVALID_FIELDID@ 0000000180005b28     libgetlocal001.obj
 0002:00000b48       ??_C@_0BL@NELIEPEC@JVMTI_ERROR_NO_MORE_FRAMES@ 0000000180005b48     libgetlocal001.obj
 0002:00000b68       ??_C@_0BJ@BDBECFDM@JVMTI_ERROR_OPAQUE_FRAME@ 0000000180005b68     libgetlocal001.obj
 0002:00000b88       ??_C@_0BK@MIIFNLOB@JVMTI_ERROR_TYPE_MISMATCH@ 0000000180005b88     libgetlocal001.obj
 0002:00000ba8       ??_C@_0BJ@HPCAOILC@JVMTI_ERROR_INVALID_SLOT@ 0000000180005ba8     libgetlocal001.obj
 0002:00000bc8       ??_C@_0BG@CHILOPNI@JVMTI_ERROR_DUPLICATE@ 0000000180005bc8     libgetlocal001.obj
 0002:00000be0       ??_C@_0BG@DIEMLHKM@JVMTI_ERROR_NOT_FOUND@ 0000000180005be0     libgetlocal001.obj
 0002:00000bf8       ??_C@_0BM@NHMCKHOB@JVMTI_ERROR_INVALID_MONITOR@ 0000000180005bf8     libgetlocal001.obj
 0002:00000c18       ??_C@_0BO@PPEDAJGL@JVMTI_ERROR_NOT_MONITOR_OWNER@ 0000000180005c18     libgetlocal001.obj
 0002:00000c38       ??_C@_0BG@FCAIPEID@JVMTI_ERROR_INTERRUPT@ 0000000180005c38     libgetlocal001.obj
 0002:00000c50       ??_C@_0CB@EGDBNKOI@JVMTI_ERROR_INVALID_CLASS_FORMA@ 0000000180005c50     libgetlocal001.obj
 0002:00000c78       ??_C@_0CG@DGKOGIAL@JVMTI_ERROR_CIRCULAR_CLASS_DEFI@ 0000000180005c78     libgetlocal001.obj
 0002:00000ca0       ??_C@_0BP@ICEALPKC@JVMTI_ERROR_FAILS_VERIFICATION@ 0000000180005ca0     libgetlocal001.obj
 0002:00000cc0       ??_C@_0DC@JDACLMIO@JVMTI_ERROR_UNSUPPORTED_REDEFIN@ 0000000180005cc0     libgetlocal001.obj
 0002:00000cf8       ??_C@_0DE@GKDKNOMJ@JVMTI_ERROR_UNSUPPORTED_REDEFIN@ 0000000180005cf8     libgetlocal001.obj
 0002:00000d30       ??_C@_0BO@LAFKIOG@JVMTI_ERROR_INVALID_TYPESTATE@ 0000000180005d30     libgetlocal001.obj
 0002:00000d50       ??_C@_0DH@INDGCLLB@JVMTI_ERROR_UNSUPPORTED_REDEFIN@ 0000000180005d50     libgetlocal001.obj
 0002:00000d88       ??_C@_0DE@NHEOMMGI@JVMTI_ERROR_UNSUPPORTED_REDEFIN@ 0000000180005d88     libgetlocal001.obj
 0002:00000dc0       ??_C@_0CA@EKPNJOEP@JVMTI_ERROR_UNSUPPORTED_VERSION@ 0000000180005dc0     libgetlocal001.obj
 0002:00000de0       ??_C@_0BN@OFFMAHHL@JVMTI_ERROR_NAMES_DONT_MATCH@ 0000000180005de0     libgetlocal001.obj
 0002:00000e00       ??_C@_0DN@HHBBLAKE@JVMTI_ERROR_UNSUPPORTED_REDEFIN@ 0000000180005e00     libgetlocal001.obj
 0002:00000e40       ??_C@_0DO@HMBGBGNA@JVMTI_ERROR_UNSUPPORTED_REDEFIN@ 0000000180005e40     libgetlocal001.obj
 0002:00000e80       ??_C@_0BP@PBECGKHJ@JVMTI_ERROR_UNMODIFIABLE_CLASS@ 0000000180005e80     libgetlocal001.obj
 0002:00000ea0       ??_C@_0BK@CANILEHF@JVMTI_ERROR_NOT_AVAILABLE@ 0000000180005ea0     libgetlocal001.obj
 0002:00000ec0       ??_C@_0CE@INJKMEFK@JVMTI_ERROR_MUST_POSSESS_CAPABI@ 0000000180005ec0     libgetlocal001.obj
 0002:00000ee8       ??_C@_0BJ@LBFPFPDM@JVMTI_ERROR_NULL_POINTER@ 0000000180005ee8     libgetlocal001.obj
 0002:00000f08       ??_C@_0BP@CHJPNNEM@JVMTI_ERROR_ABSENT_INFORMATION@ 0000000180005f08     libgetlocal001.obj
 0002:00000f28       ??_C@_0BP@OMFMNLC@JVMTI_ERROR_INVALID_EVENT_TYPE@ 0000000180005f28     libgetlocal001.obj
 0002:00000f48       ??_C@_0BN@BIBNPHHO@JVMTI_ERROR_ILLEGAL_ARGUMENT@ 0000000180005f48     libgetlocal001.obj
 0002:00000f68       ??_C@_0BK@KKNDHDCE@JVMTI_ERROR_NATIVE_METHOD@ 0000000180005f68     libgetlocal001.obj
 0002:00000f88       ??_C@_0BK@PMKCFHAE@JVMTI_ERROR_OUT_OF_MEMORY@ 0000000180005f88     libgetlocal001.obj
 0002:00000fa8       ??_C@_0BK@NNJBDMNB@JVMTI_ERROR_ACCESS_DENIED@ 0000000180005fa8     libgetlocal001.obj
 0002:00000fc8       ??_C@_0BI@GHECLMNC@JVMTI_ERROR_WRONG_PHASE@ 0000000180005fc8     libgetlocal001.obj
 0002:00000fe0       ??_C@_0BF@OLIHJOII@JVMTI_ERROR_INTERNAL@ 0000000180005fe0     libgetlocal001.obj
 0002:00000ff8       ??_C@_0BO@EOHGKJHI@JVMTI_ERROR_UNATTACHED_THREAD@ 0000000180005ff8     libgetlocal001.obj
 0002:00001018       ??_C@_0CA@LKHFDACL@JVMTI_ERROR_INVALID_ENVIRONMENT@ 0000000180006018     libgetlocal001.obj
 0002:00001038       ??_C@_0BA@MMFHLOKK@?$DMunknown?5error?$DO@ 0000000180006038     libgetlocal001.obj
 0002:00001048       ??_C@_0CF@CBHOKDB@throwable?5?$DN?5jni?9?$DOExceptionOccur@ 0000000180006048     libgetlocal001.obj
 0002:00001070       ??_C@_03OFAPEBGM@?$CFs?6@  0000000180006070     libgetlocal001.obj
 0002:00001078       ??_C@_0DM@LPIGEGNJ@s?2test?2hotspot?2jtreg?2vmTestbase@ 0000000180006078     libgetlocal001.obj
 0002:000010b8       ??_C@_0CC@NFCNPEPK@Exception?5in?5JNI?5call?5?$CIcleared?$CJ@ 00000001800060b8     libgetlocal001.obj
 0002:000010e0       ??_C@_0BJ@IBAKFIKF@jni?9?$DOExceptionDescribe?$CI?$CJ@ 00000001800060e0     libgetlocal001.obj
 0002:00001100       ??_C@_0BG@GGKALKMH@jni?9?$DOExceptionClear?$CI?$CJ@ 0000000180006100     libgetlocal001.obj
 0002:00001118       ??_C@_0CF@JMGFGJLJ@?$CD?5?5?5verified?5JNI?5assertion?5is?5F@ 0000000180006118     libgetlocal001.obj
 0002:00001140       ??_C@_0CB@MLNJNCLJ@?5?5jvmti?5error?3?5code?$DN?$CFd?0?5name?$DN?$CFs@ 0000000180006140     libgetlocal001.obj
 0002:00001168       ??_C@_0CD@OHBGDKMK@?$CD?5?5?5jvmti?5error?3?5code?$DN?$CFd?0?5name?$DN@ 0000000180006168     libgetlocal001.obj
 0002:00001190       ??_C@_0CG@JNNCGPHB@?$CD?5?5?5error?5expected?3?5code?$DN?$CFd?0?5na@ 0000000180006190     libgetlocal001.obj
 0002:000011c0       ??_C@_0EB@IMGKPCGE@?$CIstr_obj?5?$DN?5jni?9?$DONewStringUTF?$CIco@ 00000001800061c0     libgetlocal001.obj
 0002:00001210       ??_C@_0EA@HFOGGBCC@s?2test?2hotspot?2jtreg?2vmTestbase@ 0000000180006210     libgetlocal001.obj
 0002:00001250       ??_C@_0CO@HJKAMPK@?$CIGetFrameLocation?$CJ?5unexpected?5e@ 0000000180006250     libgetlocal001.obj
 0002:00001280       ??_C@_05KKCIMGE@error@     0000000180006280     libgetlocal001.obj
 0002:00001290       ??_C@_0EA@PNBCDMOA@s?2test?2hotspot?2jtreg?2vmTestbase@ 0000000180006290     libgetlocal001.obj
 0002:000012d0       ??_C@_0DI@ILAHDLMP@?$CI?$CKagentThreadProc?$CJ?$CIjvmti_env?0?5a@ 00000001800062d0     libgetlocal001.obj
 0002:00001308       ??_C@_0BD@KDBALNLB@JVMTI?5agent?5thread@ 0000000180006308     libgetlocal001.obj
 0002:00001320       ??_C@_0BB@NOKBFPFO@java?1lang?1Thread@ 0000000180006320     libgetlocal001.obj
 0002:00001334       ??_C@_06FALKBLGB@?$DMinit?$DO@ 0000000180006334     libgetlocal001.obj
 0002:00001340       ??_C@_0BG@IKDDPPGD@?$CILjava?1lang?1String?$DL?$CJV@ 0000000180006340     libgetlocal001.obj
 0002:00001360       ??_C@_0EB@IFJBFEKC@?$CIthreadClass?5?$DN?5jni_env?9?$DOFindCla@ 0000000180006360     libgetlocal001.obj
 0002:000013b0       ??_C@_0GF@FGFIBKKL@?$CIthreadCtor?5?$DN?5jni_env?9?$DOGetMetho@ 00000001800063b0     libgetlocal001.obj
 0002:00001418       ??_C@_0DN@NCPDJLOG@?$CIthreadName?5?$DN?5jni_env?9?$DONewStrin@ 0000000180006418     libgetlocal001.obj
 0002:00001460       ??_C@_0FE@PFKODBGC@?$CIthreadObject?5?$DN?5jni_env?9?$DONewObj@ 0000000180006460     libgetlocal001.obj
 0002:000014c0       ??_C@_0ED@HOBAHHJI@?$CIthreadGlobalRef?5?$DN?5jni_env?9?$DONew@ 00000001800064c0     libgetlocal001.obj
 0002:00001510       ??_C@_0FN@HNJJAHFC@jvmti_env?9?$DORunAgentThread?$CIagent@ 0000000180006510     libgetlocal001.obj
 0002:00001570       ??_C@_0EA@MOJDNKDF@Debuggee?5status?5sync?5aborted?5be@ 0000000180006570     libgetlocal001.obj
 0002:000015b0       ??_C@_0EA@EEOEJAEN@status?5?$DN?5syncDebuggeeStatus?$CIjni@ 00000001800065b0     libgetlocal001.obj
 0002:000015f0       ??_C@_0BL@JBCFNBMB@nsk_jvmti_resetAgentData?$CI?$CJ@ 00000001800065f0     libgetlocal001.obj
 0002:00001610       ??_C@_0EL@LPBEELIP@s?2test?2hotspot?2jtreg?2vmTestbase@ 0000000180006610     libgetlocal001.obj
 0002:00001660       ??_C@_0CK@JDAMFDMJ@jvmti?9?$DOSetTag?$CIo?0?5tag?$CJ?5?$DN?$DN?5JVMTI_@ 0000000180006660     libgetlocal001.obj
 0002:00001690       ??_C@_0CC@DAMNHKNI@Can?8t?5set?5tag?5?$CFli?5for?5object?5?$CFl@ 0000000180006690     libgetlocal001.obj
 0002:000016b8       ??_C@_0DL@HAJPNKEF@jvmti?9?$DOGetObjectHashCode?$CIo?0?5?$CGha@ 00000001800066b8     libgetlocal001.obj
 0002:000016f8       ??_C@_0BL@JFPIEOBF@Can?8t?5get?5hash?5object?5?$CFlx?6@ 00000001800066f8     libgetlocal001.obj
 0002:00001718       ??_C@_0BG@DICPHBKN@setTag?3?5?$CF08x?5?$DM?9?5?$CF?53li@ 0000000180006718     libgetlocal001.obj
 0002:00001730       ??_C@_0DH@FCEEBDMJ@?$CIs?5?$DN?5jni?9?$DOGetStringUTFChars?$CIsIn@ 0000000180006730     libgetlocal001.obj
 0002:00001768       ??_C@_0BJ@OKKGHDCN@Can?8t?5get?5string?5at?5?$CF?$CDp?6@ 0000000180006768     libgetlocal001.obj
 0002:00001788       ??_C@_0BP@EKFLGGFJ@Can?8t?5get?5string?5at?5?$CF?$CDp?3?5null?6@ 0000000180006788     libgetlocal001.obj
 0002:000017a8       ??_C@_06ICODBHCL@?5?1?1?5?$CFs@ 00000001800067a8     libgetlocal001.obj
 0002:000017b0       ??_C@_0DB@KGFPLEGO@?$CIr?5?$DN?5jvmti?9?$DOGetTag?$CIo?0?5?$CGtag?$CJ?$CJ?5?$DN?$DN@ 00000001800067b0     libgetlocal001.obj
 0002:000017e8       ??_C@_0CO@PDAGBCGJ@Can?8t?5GetTag?5for?5object?5?$CFlx?4?5Re@ 00000001800067e8     libgetlocal001.obj
 0002:00001818       ??_C@_0CH@HPEODOHC@TEST_BUG?3?5Max?4?5number?5of?5refs?5r@ 0000000180006818     libgetlocal001.obj
 0002:00001840       ??_C@_0DI@PHFCABIM@?$CIr?5?$DN?5jvmti?9?$DOGetTag?$CIfrom?0?5?$CGtagFr@ 0000000180006840     libgetlocal001.obj
 0002:00001878       ??_C@_0DI@MDEGFNKD@TEST_BUG?3?5Can?8t?5GetTag?5for?5obje@ 0000000180006878     libgetlocal001.obj
 0002:000018b0       ??_C@_0DE@MLELJAHM@?$CIr?5?$DN?5jvmti?9?$DOGetTag?$CIto?0?5?$CGtagTo?$CJ?$CJ@ 00000001800068b0     libgetlocal001.obj
 0002:000018e4       ??_C@_03GAEACAIP@?$CI?$CJV@ 00000001800068e4     libgetlocal001.obj
 0002:000018e8       ??_C@_01HHGOMJKL@l@        00000001800068e8     libgetlocal001.obj
 0002:000018f0       ??_C@_0CM@GFMFEJIC@?$CIGetLocalLong?$CD1?$CJ?5unexpected?5err@ 00000001800068f0     libgetlocal001.obj
 0002:0000191c       ??_C@_01INIBCBCB@f@        000000018000691c     libgetlocal001.obj
 0002:00001920       ??_C@_0CN@IAKHFLPE@?$CIGetLocalFloat?$CD1?$CJ?5unexpected?5er@ 0000000180006920     libgetlocal001.obj
 0002:00001950       ??_C@_01LPLHEDKD@d@        0000000180006950     libgetlocal001.obj
 0002:00001958       ??_C@_0CO@OKMCHLMD@?$CIGetLocalDouble?$CD1?$CJ?5unexpected?5e@ 0000000180006958     libgetlocal001.obj
 0002:00001988       ??_C@_0DG@CDNAEEAM@One?5of?5values?5retrieved?5by?5GetL@ 0000000180006988     libgetlocal001.obj
 0002:000019c0       ??_C@_0DI@OMCHNNMD@?5?5?5?5actual?3?5long?5?$DN?50x?$CF08x?$CF08x?0?5@ 00000001800069c0     libgetlocal001.obj
 0002:000019f8       ??_C@_0DI@DMPGGKNA@?5?5expected?3?5long?5?$DN?50x?$CF08x?$CF08x?0?5@ 00000001800069f8     libgetlocal001.obj
 0002:00001a30       ??_C@_02IBOFNBPA@i1@       0000000180006a30     libgetlocal001.obj
 0002:00001a38       ??_C@_0CN@LKEAKFLF@?$CIGetLocalInt?$CD2i1?$CJ?5unexpected?5er@ 0000000180006a38     libgetlocal001.obj
 0002:00001a68       ??_C@_02KKMIICDD@i2@       0000000180006a68     libgetlocal001.obj
 0002:00001a70       ??_C@_0CN@POOBIAKN@?$CIGetLocalInt?$CD2i2?$CJ?5unexpected?5er@ 0000000180006a70     libgetlocal001.obj
 0002:00001aa0       ??_C@_02LDNDLDHC@i3@       0000000180006aa0     libgetlocal001.obj
 0002:00001aa8       ??_C@_0CN@MCIBGDKF@?$CIGetLocalInt?$CD2i3?$CJ?5unexpected?5er@ 0000000180006aa8     libgetlocal001.obj
 0002:00001ad8       ??_C@_02PMJCCFLF@i4@       0000000180006ad8     libgetlocal001.obj
 0002:00001ae0       ??_C@_0CN@HHKDMKJN@?$CIGetLocalInt?$CD2i4?$CJ?5unexpected?5er@ 0000000180006ae0     libgetlocal001.obj
 0002:00001b10       ??_C@_02OFIJBEPE@i5@       0000000180006b10     libgetlocal001.obj
 0002:00001b18       ??_C@_0CN@ELMDCJJF@?$CIGetLocalInt?$CD2i5?$CJ?5unexpected?5er@ 0000000180006b18     libgetlocal001.obj
 0002:00001b48       ??_C@_0DI@EMNCCKNF@One?5of?5values?5retrieved?5by?5GetL@ 0000000180006b48     libgetlocal001.obj
 0002:00001b80       ??_C@_0DM@KKOAPEO@?5?5?5?5actual?3?5int?$DN?$CFd?0?5short?$DN?$CFd?0?5c@ 0000000180006b80     libgetlocal001.obj
 0002:00001bc0       ??_C@_0DM@JGODDJCA@?5?5expected?3?5int?$DN?$CFd?0?5short?$DN?$CFd?0?5c@ 0000000180006bc0     libgetlocal001.obj
 0002:00001bfc       ??_C@_03DAPANPEK@ob1@      0000000180006bfc     libgetlocal001.obj
 0002:00001c00       ??_C@_0CO@MIEHPDMF@?$CIGetLocalObject?$CD1?$CJ?5unexpected?5e@ 0000000180006c00     libgetlocal001.obj
 0002:00001c30       ??_C@_0DF@BMPOKPHD@?$CIGetMethodDeclaringClass?$CJ?5unexp@ 0000000180006c30     libgetlocal001.obj
 0002:00001c68       ??_C@_01JPJNBJEM@I@        0000000180006c68     libgetlocal001.obj
 0002:00001c6c       ??_C@_03IAKKBENL@fld@      0000000180006c6c     libgetlocal001.obj
 0002:00001c70       ??_C@_0CK@GJEJLGNL@Cannot?5find?5ID?5for?5?$CCfld?$CC?5field?5@ 0000000180006c70     libgetlocal001.obj
 0002:00001c9c       ??_C@_03BLNNIMIJ@ob2@      0000000180006c9c     libgetlocal001.obj
 0002:00001ca0       ??_C@_0CO@IMOGNGNN@?$CIGetLocalObject?$CD2?$CJ?5unexpected?5e@ 0000000180006ca0     libgetlocal001.obj
 0002:00001cd0       ??_C@_0DM@HILNALFB@One?5of?5objects?5retrieved?5by?5Get@ 0000000180006cd0     libgetlocal001.obj
 0002:00001d10       ??_C@_0CK@HHAHCDMD@?5?5?5?5actual?3?5fldVal?5?$DN?5?$CFd?0?5int?4ar@ 0000000180006d10     libgetlocal001.obj
 0002:00001d40       ??_C@_0CK@IJHAFGFH@?5?5expected?3?5fldVal?5?$DN?5?$CFd?0?5int?4ar@ 0000000180006d40     libgetlocal001.obj
 0002:00001d70       ??_C@_0CN@PDAPLCIK@?$CIGetLocalInt?$CD4i1?$CJ?5unexpected?5er@ 0000000180006d70     libgetlocal001.obj
 0002:00001da0       ??_C@_0CN@LHKOJHJC@?$CIGetLocalInt?$CD4i2?$CJ?5unexpected?5er@ 0000000180006da0     libgetlocal001.obj
 0002:00001dd0       ??_C@_0CN@ILMOHEJK@?$CIGetLocalInt?$CD4i3?$CJ?5unexpected?5er@ 0000000180006dd0     libgetlocal001.obj
 0002:00001e00       ??_C@_0CN@DOOMNNKC@?$CIGetLocalInt?$CD4i4?$CJ?5unexpected?5er@ 0000000180006e00     libgetlocal001.obj
 0002:00001e30       ??_C@_01OJONOECF@b@        0000000180006e30     libgetlocal001.obj
 0002:00001e38       ??_C@_0CM@DACCKGKJ@?$CIGetLocalInt?$CD4b?$CJ?5unexpected?5err@ 0000000180006e38     libgetlocal001.obj
 0002:00001e68       ??_C@_0CM@KICGCGKK@?$CIGetLocalLong?$CD4?$CJ?5unexpected?5err@ 0000000180006e68     libgetlocal001.obj
 0002:00001e98       ??_C@_0CN@ENEEDENM@?$CIGetLocalFloat?$CD4?$CJ?5unexpected?5er@ 0000000180006e98     libgetlocal001.obj
 0002:00001ec8       ??_C@_0CO@CHCBBEOL@?$CIGetLocalDouble?$CD4?$CJ?5unexpected?5e@ 0000000180006ec8     libgetlocal001.obj
 0002:00001ef8       ??_C@_0DI@MCMPHCDB@One?5of?5values?5retrieved?5by?5GetL@ 0000000180006ef8     libgetlocal001.obj
 0002:00001f30       ??_C@_0DI@CNCJBCMM@?5?5?5?5?5?5?5?5?5?5?5?5long?5?$DN?50x?$CF08x?$CF08x?0?5@ 0000000180006f30     libgetlocal001.obj
 0002:00001f68       ??_C@_0DF@NAAAGOJC@?$CIGetLocalVariableTable?$CD1?$CJ?5unexp@ 0000000180006f68     libgetlocal001.obj
 0002:00001fa0       ??_C@_0BC@LJPAILDM@?$DO?$DO?$DO?5exit?3?5meth01?6@ 0000000180006fa0     libgetlocal001.obj
 0002:00001fb8       ??_C@_0BC@LLLGDFGF@?$DO?$DO?$DO?5exit?3?5meth02?6@ 0000000180006fb8     libgetlocal001.obj
 0002:00001fd0       ??_C@_0BC@LKHEFPFC@?$DO?$DO?$DO?5exit?3?5meth03?6@ 0000000180006fd0     libgetlocal001.obj
 0002:00001fe8       ??_C@_0BC@LPDLEJNH@?$DO?$DO?$DO?5exit?3?5meth04?6@ 0000000180006fe8     libgetlocal001.obj
 0002:00002000       ??_C@_0DF@JEKBELIK@?$CIGetLocalVariableTable?$CD2?$CJ?5unexp@ 0000000180007000     libgetlocal001.obj
 0002:00002038       ??_C@_0BA@HDKOOOEO@?$DO?$DO?$DO?5bp?3?5meth01?6@ 0000000180007038     libgetlocal001.obj
 0002:00002048       ??_C@_0BA@HBOIFABH@?$DO?$DO?$DO?5bp?3?5meth02?6@ 0000000180007048     libgetlocal001.obj
 0002:00002058       ??_C@_0BA@HACKDKCA@?$DO?$DO?$DO?5bp?3?5meth03?6@ 0000000180007058     libgetlocal001.obj
 0002:00002068       ??_C@_0BA@HFGFCMKF@?$DO?$DO?$DO?5bp?3?5meth04?6@ 0000000180007068     libgetlocal001.obj
 0002:00002078       ??_C@_0CM@EGMIFBJC@ERROR?3?5didn?8t?5know?5where?5we?5got@ 0000000180007078     libgetlocal001.obj
 0002:000020a8       ??_C@_09OPJEJKBL@printdump@ 00000001800070a8     libgetlocal001.obj
 0002:000020b8       ??_C@_0CK@DEFLIKCM@Wrong?5result?5of?5a?5valid?5call?5to@ 00000001800070b8     libgetlocal001.obj
 0002:000020e8       ??_C@_0DG@LAJPGIIE@?$CIGetPotentialCapabilities?$CJ?5unex@ 00000001800070e8     libgetlocal001.obj
 0002:00002120       ??_C@_0CN@LKPEOJPO@?$CIAddCapabilities?$CJ?5unexpected?5er@ 0000000180007120     libgetlocal001.obj
 0002:00002150       ??_C@_0CN@BCCBOHCH@?$CIGetCapabilities?$CJ?5unexpected?5er@ 0000000180007150     libgetlocal001.obj
 0002:00002180       ??_C@_0DH@HAICLNGL@Warning?3?5Access?5to?5local?5variab@ 0000000180007180     libgetlocal001.obj
 0002:000021b8       ??_C@_0CP@IMINGNLL@?$CISetEventCallbacks?$CJ?5unexpected?5@ 00000001800071b8     libgetlocal001.obj
 0002:000021e8       ??_C@_0DM@HLHCJLLD@Warning?3?5Breakpoint?5or?5MethodEx@ 00000001800071e8     libgetlocal001.obj
 0002:00002224       ??_C@_03BILEFAFM@?$CI?$CJD@ 0000000180007224     libgetlocal001.obj
 0002:00002228       ??_C@_06MADNOIIM@meth01@   0000000180007228     libgetlocal001.obj
 0002:00002230       ??_C@_04PFANPMCN@?$CII?$CJV@ 0000000180007230     libgetlocal001.obj
 0002:00002238       ??_C@_06OLBALLEP@meth02@   0000000180007238     libgetlocal001.obj
 0002:00002240       ??_C@_0CM@NKDNGHBN@?$CILnsk?1jvmti?1GetLocalVariable?1ge@ 0000000180007240     libgetlocal001.obj
 0002:0000226c       ??_C@_06PCALIKAO@meth03@   000000018000726c     libgetlocal001.obj
 0002:00002278       ??_C@_0M@KJJOHAPG@?$CIIJSDCFBZ?$CJV@ 0000000180007278     libgetlocal001.obj
 0002:00002284       ??_C@_06LNEKBMMJ@meth04@   0000000180007284     libgetlocal001.obj
 0002:00002290       ??_C@_0L@GIHILDI@checkPoint@ 0000000180007290     libgetlocal001.obj
 0002:000022a0       ??_C@_0CE@HCBNHAFL@Cannot?5find?5Method?5ID?5for?5a?5met@ 00000001800072a0     libgetlocal001.obj
 0002:000022c8       ??_C@_0CN@GHJIKGLO@Failed?5to?5enable?5METHOD_EXIT?5ev@ 00000001800072c8     libgetlocal001.obj
 0002:000022f8       ??_C@_0CD@GGHKKOMC@Failed?5to?5SetBreakpoint?3?5err?5?$DN?5@ 00000001800072f8     libgetlocal001.obj
 0002:00002320       ??_C@_0CM@NEGFNKGE@Failed?5to?5enable?5BREAKPOINT?5eve@ 0000000180007320     libgetlocal001.obj
 0002:00002350       __real@4018000000000000    0000000180007350     libgetlocal001.obj
 0002:00002358       __real@401c000000000000    0000000180007358     libgetlocal001.obj
 0002:00002360       __real@40c00000            0000000180007360     libgetlocal001.obj
 0002:00002380       ??_C@_1EC@JIJBPKFM@?$AAa?$AAp?$AAi?$AA?9?$AAm?$AAs?$AA?9?$AAw?$AAi?$AAn?$AA?9?$AAc?$AAo?$AAr?$AAe@ 0000000180007380     MSVCRT:thread_safe_statics.obj
 0002:000023c8       ??_C@_1BK@MGMFAEKH@?$AAk?$AAe?$AAr?$AAn?$AAe?$AAl?$AA3?$AA2?$AA?4?$AAd?$AAl?$AAl@ 00000001800073c8     MSVCRT:thread_safe_statics.obj
 0002:000023e8       ??_C@_0BJ@JEBJOJFJ@SleepConditionVariableCS@ 00000001800073e8     MSVCRT:thread_safe_statics.obj
 0002:00002408       ??_C@_0BJ@PGPPEPCC@WakeAllConditionVariable@ 0000000180007408     MSVCRT:thread_safe_statics.obj
 0002:00002428       _pDefaultRawDllMain        0000000180007428     MSVCRT:dll_dllmain.obj
 0002:00002428       _pRawDllMain               0000000180007428     MSVCRT:dll_dllmain.obj
 0002:00002430       __xmm@ffffffffffffffffffffffffffffffff 0000000180007430     MSVCRT:utility.obj
 0002:00002440       _load_config_used          0000000180007440     MSVCRT:loadcfg.obj
 0002:00002600       _tls_used                  0000000180007600     MSVCRT:tlssup.obj
 0002:00002628       __volatile_metadata        0000000180007628     <linker-defined>
 0002:000029f0       __rtc_iaa                  00000001800079f0     MSVCRT:initsect.obj
 0002:000029f8       __rtc_izz                  00000001800079f8     MSVCRT:initsect.obj
 0002:00002a00       __rtc_taa                  0000000180007a00     MSVCRT:initsect.obj
 0002:00002a08       __rtc_tzz                  0000000180007a08     MSVCRT:initsect.obj
 0002:00002a10       _tls_start                 0000000180007a10     MSVCRT:tlssup.obj
 0002:00002a14       _Init_thread_epoch         0000000180007a14     MSVCRT:thread_safe_statics.obj
 0002:00002a18       _tls_end                   0000000180007a18     MSVCRT:tlssup.obj
 0002:00003180       __IMPORT_DESCRIPTOR_KERNEL32 0000000180008180     kernel32:KERNEL32.dll
 0002:00003194       __IMPORT_DESCRIPTOR_VCRUNTIME140 0000000180008194     vcruntime:VCRUNTIME140.dll
 0002:000031a8       __IMPORT_DESCRIPTOR_api-ms-win-crt-runtime-l1-1-0 00000001800081a8     ucrt:api-ms-win-crt-runtime-l1-1-0.dll
 0002:000031bc       __IMPORT_DESCRIPTOR_api-ms-win-crt-stdio-l1-1-0 00000001800081bc     ucrt:api-ms-win-crt-stdio-l1-1-0.dll
 0002:000031d0       __IMPORT_DESCRIPTOR_api-ms-win-crt-string-l1-1-0 00000001800081d0     ucrt:api-ms-win-crt-string-l1-1-0.dll
 0002:000031e4       __NULL_IMPORT_DESCRIPTOR   00000001800081e4     kernel32:KERNEL32.dll
 0003:00000030       _Init_global_epoch         0000000180009030     MSVCRT:thread_safe_statics.obj
 0003:00000040       __security_cookie          0000000180009040     MSVCRT:gs_cookie.obj
 0003:00000048       __security_cookie_complement 0000000180009048     MSVCRT:gs_cookie.obj
 0003:00000050       _fltused                   0000000180009050     MSVCRT:fltused.obj
 0003:00000054       __scrt_native_dllmain_reason 0000000180009054     MSVCRT:utility.obj
 0003:00000058       __isa_available            0000000180009058     MSVCRT:cpu_disp.obj
 0003:0000005c       __isa_enabled              000000018000905c     MSVCRT:cpu_disp.obj
 0003:00000060       __memset_fast_string_threshold 0000000180009060     MSVCRT:cpu_disp.obj
 0003:00000068       __memset_nt_threshold      0000000180009068     MSVCRT:cpu_disp.obj
 0003:00000070       __scrt_ucrt_dll_is_in_use  0000000180009070     MSVCRT:ucrt_stubs.obj
 0003:00000080       g_wrongHeapCallbacks       0000000180009080     libgetlocal001.obj
 0003:00000100       g_szTagInfo                0000000180009100     libgetlocal001.obj
 0003:00002040       g_tagFlags                 000000018000b040     libgetlocal001.obj
 0003:00002428       g_refsToVerifyCnt          000000018000b428     libgetlocal001.obj
 0003:0000242c       g_fakeUserData             000000018000b42c     libgetlocal001.obj
 0003:00002430       g_tagVisitCount            000000018000b430     libgetlocal001.obj
 0003:000033d0       g_refsToVerify             000000018000c3d0     libgetlocal001.obj
 0003:0001aad0       g_userDataError            0000000180023ad0     libgetlocal001.obj
 0003:0001ade8       ?_OptionsStorage@?1??__local_stdio_printf_options@@9@4_KA 0000000180023de8     libgetlocal001.obj
 0003:0001b3a8       _tls_index                 00000001800243a8     MSVCRT:tlssup.obj
 0003:0001b3b0       __scrt_current_native_startup_state 00000001800243b0     MSVCRT:utility.obj
 0003:0001b3b8       __scrt_native_startup_lock 00000001800243b8     MSVCRT:utility.obj
 0003:0001b3f8       __scrt_debugger_hook_flag  00000001800243f8     MSVCRT:utility_desktop.obj
 0003:0001b400       ?__type_info_root_node@@3U__type_info_node@@A 0000000180024400     MSVCRT:tncleanup.obj
 0003:0001b410       ?_OptionsStorage@?1??__local_stdio_scanf_options@@9@4_KA 0000000180024410     MSVCRT:default_local_stdio_options.obj
 0003:0001b418       __favor                    0000000180024418     MSVCRT:cpu_disp.obj
 0003:0001b420       __dyn_tls_init_callback    0000000180024420     <common>

 entry point at        0001:00003270

 Static symbols

 0000:fffd9000       .debug$S                   0000000180000000     getlocal001.exp
 0000:fffd9000       .debug$S                   0000000180000000     vcruntime:VCRUNTIME140.dll
 0000:fffd9000       .debug$S                   0000000180000000     vcruntime:VCRUNTIME140.dll
 0000:fffd9000       .debug$S                   0000000180000000     vcruntime:VCRUNTIME140.dll
 0000:fffd9000       .debug$S                   0000000180000000     vcruntime:VCRUNTIME140.dll
 0000:fffd9000       .debug$S                   0000000180000000     vcruntime:VCRUNTIME140.dll
 0000:fffd9000       .debug$S                   0000000180000000     vcruntime:VCRUNTIME140.dll
 0000:fffd9000       .debug$S                   0000000180000000     vcruntime:VCRUNTIME140.dll
 0000:fffd9000       .debug$S                   0000000180000000     ucrt:api-ms-win-crt-convert-l1-1-0.dll
 0002:ffffb000       .idata$6                   0000000180000000     ucrt:api-ms-win-crt-convert-l1-1-0.dll
 0000:fffd9000       .debug$S                   0000000180000000     ucrt:api-ms-win-crt-heap-l1-1-0.dll
 0000:fffd9000       .debug$S                   0000000180000000     ucrt:api-ms-win-crt-heap-l1-1-0.dll
 0000:fffd9000       .debug$S                   0000000180000000     ucrt:api-ms-win-crt-heap-l1-1-0.dll
 0000:fffd9000       .debug$S                   0000000180000000     ucrt:api-ms-win-crt-heap-l1-1-0.dll
 0002:ffffb000       .idata$6                   0000000180000000     ucrt:api-ms-win-crt-heap-l1-1-0.dll
 0000:fffd9000       .debug$S                   0000000180000000     ucrt:api-ms-win-crt-runtime-l1-1-0.dll
 0000:fffd9000       .debug$S                   0000000180000000     ucrt:api-ms-win-crt-runtime-l1-1-0.dll
 0000:fffd9000       .debug$S                   0000000180000000     ucrt:api-ms-win-crt-runtime-l1-1-0.dll
 0000:fffd9000       .debug$S                   0000000180000000     ucrt:api-ms-win-crt-runtime-l1-1-0.dll
 0000:fffd9000       .debug$S                   0000000180000000     ucrt:api-ms-win-crt-runtime-l1-1-0.dll
 0000:fffd9000       .debug$S                   0000000180000000     ucrt:api-ms-win-crt-runtime-l1-1-0.dll
 0000:fffd9000       .debug$S                   0000000180000000     ucrt:api-ms-win-crt-runtime-l1-1-0.dll
 0000:fffd9000       .debug$S                   0000000180000000     ucrt:api-ms-win-crt-runtime-l1-1-0.dll
 0000:fffd9000       .debug$S                   0000000180000000     ucrt:api-ms-win-crt-runtime-l1-1-0.dll
 0000:fffd9000       .debug$S                   0000000180000000     ucrt:api-ms-win-crt-runtime-l1-1-0.dll
 0000:fffd9000       .debug$S                   0000000180000000     ucrt:api-ms-win-crt-runtime-l1-1-0.dll
 0000:fffd9000       .debug$S                   0000000180000000     ucrt:api-ms-win-crt-runtime-l1-1-0.dll
 0000:fffd9000       .debug$S                   0000000180000000     ucrt:api-ms-win-crt-runtime-l1-1-0.dll
 0000:fffd9000       .debug$S                   0000000180000000     ucrt:api-ms-win-crt-runtime-l1-1-0.dll
 0000:fffd9000       .debug$S                   0000000180000000     ucrt:api-ms-win-crt-runtime-l1-1-0.dll
 0000:fffd9000       .debug$S                   0000000180000000     ucrt:api-ms-win-crt-runtime-l1-1-0.dll
 0000:fffd9000       .debug$S                   0000000180000000     ucrt:api-ms-win-crt-stdio-l1-1-0.dll
 0000:fffd9000       .debug$S                   0000000180000000     ucrt:api-ms-win-crt-stdio-l1-1-0.dll
 0000:fffd9000       .debug$S                   0000000180000000     ucrt:api-ms-win-crt-stdio-l1-1-0.dll
 0000:fffd9000       .debug$S                   0000000180000000     ucrt:api-ms-win-crt-stdio-l1-1-0.dll
 0000:fffd9000       .debug$S                   0000000180000000     ucrt:api-ms-win-crt-stdio-l1-1-0.dll
 0000:fffd9000       .debug$S                   0000000180000000     ucrt:api-ms-win-crt-stdio-l1-1-0.dll
 0000:fffd9000       .debug$S                   0000000180000000     ucrt:api-ms-win-crt-stdio-l1-1-0.dll
 0000:fffd9000       .debug$S                   0000000180000000     ucrt:api-ms-win-crt-stdio-l1-1-0.dll
 0000:fffd9000       .debug$S                   0000000180000000     ucrt:api-ms-win-crt-stdio-l1-1-0.dll
 0000:fffd9000       .debug$S                   0000000180000000     ucrt:api-ms-win-crt-stdio-l1-1-0.dll
 0000:fffd9000       .debug$S                   0000000180000000     ucrt:api-ms-win-crt-string-l1-1-0.dll
 0000:fffd9000       .debug$S                   0000000180000000     ucrt:api-ms-win-crt-string-l1-1-0.dll
 0000:fffd9000       .debug$S                   0000000180000000     ucrt:api-ms-win-crt-string-l1-1-0.dll
 0000:fffd9000       .debug$S                   0000000180000000     ucrt:api-ms-win-crt-string-l1-1-0.dll
 0000:fffd9000       .debug$S                   0000000180000000     ucrt:api-ms-win-crt-string-l1-1-0.dll
 0000:fffd9000       .debug$S                   0000000180000000     ucrt:api-ms-win-crt-string-l1-1-0.dll
 0000:fffd9000       .debug$S                   0000000180000000     ucrt:api-ms-win-crt-string-l1-1-0.dll
 0000:fffd9000       .debug$S                   0000000180000000     ucrt:api-ms-win-crt-string-l1-1-0.dll
 0000:fffd9000       .debug$S                   0000000180000000     kernel32:KERNEL32.dll
 0000:fffd9000       .debug$S                   0000000180000000     kernel32:KERNEL32.dll
 0000:fffd9000       .debug$S                   0000000180000000     kernel32:KERNEL32.dll
 0000:fffd9000       .debug$S                   0000000180000000     kernel32:KERNEL32.dll
 0000:fffd9000       .debug$S                   0000000180000000     kernel32:KERNEL32.dll
 0000:fffd9000       .debug$S                   0000000180000000     kernel32:KERNEL32.dll
 0000:fffd9000       .debug$S                   0000000180000000     kernel32:KERNEL32.dll
 0000:fffd9000       .debug$S                   0000000180000000     kernel32:KERNEL32.dll
 0000:fffd9000       .debug$S                   0000000180000000     kernel32:KERNEL32.dll
 0000:fffd9000       .debug$S                   0000000180000000     kernel32:KERNEL32.dll
 0000:fffd9000       .debug$S                   0000000180000000     kernel32:KERNEL32.dll
 0000:fffd9000       .debug$S                   0000000180000000     kernel32:KERNEL32.dll
 0000:fffd9000       .debug$S                   0000000180000000     kernel32:KERNEL32.dll
 0000:fffd9000       .debug$S                   0000000180000000     kernel32:KERNEL32.dll
 0000:fffd9000       .debug$S                   0000000180000000     kernel32:KERNEL32.dll
 0000:fffd9000       .debug$S                   0000000180000000     kernel32:KERNEL32.dll
 0000:fffd9000       .debug$S                   0000000180000000     kernel32:KERNEL32.dll
 0000:fffd9000       .debug$S                   0000000180000000     kernel32:KERNEL32.dll
 0000:fffd9000       .debug$S                   0000000180000000     kernel32:KERNEL32.dll
 0000:fffd9000       .debug$S                   0000000180000000     kernel32:KERNEL32.dll
 0000:fffd9000       .debug$S                   0000000180000000     kernel32:KERNEL32.dll
 0000:fffd9000       .debug$S                   0000000180000000     kernel32:KERNEL32.dll
 0000:fffd9000       .debug$S                   0000000180000000     kernel32:KERNEL32.dll
 0000:fffd9000       .debug$S                   0000000180000000     kernel32:KERNEL32.dll
 0000:fffd9000       .debug$S                   0000000180000000     kernel32:KERNEL32.dll
 0000:fffd9000       .debug$S                   0000000180000000     kernel32:KERNEL32.dll
 0000:fffd9000       .debug$S                   0000000180000000     kernel32:KERNEL32.dll
 0000:fffd9000       .debug$S                   0000000180000000     kernel32:KERNEL32.dll
 0001:0000141c       addRefToVerify             000000018000241c f   libgetlocal001.obj
 0001:00001490       agentThreadWrapper         0000000180002490 f   libgetlocal001.obj
 0001:00002158       file_basename              0000000180003158 f   libgetlocal001.obj
 0001:00002780       startAgentThreadWrapper    0000000180003780 f   libgetlocal001.obj
 0001:00002aac       syncDebuggeeStatus         0000000180003aac f   libgetlocal001.obj
 0001:00002d34       capture_previous_context   0000000180003d34 f   MSVCRT:gs_report.obj
 0001:00002da8       ?__scrt_initialize_thread_safe_statics@@YAHXZ 0000000180003da8 f   MSVCRT:thread_safe_statics.obj
 0001:00002e78       ?__scrt_uninitialize_thread_safe_statics@@YAXXZ 0000000180003e78 f   MSVCRT:thread_safe_statics.obj
 0001:00002f20       $$000000                   0000000180003f20     MSVCRT:amdsecgs.obj
 0001:00002f50       ?dllmain_crt_dispatch@@YAHQEAUHINSTANCE__@@KQEAX@Z 0000000180003f50 f   MSVCRT:dll_dllmain.obj
 0001:00002fa0       ?dllmain_crt_process_attach@@YAHQEAUHINSTANCE__@@QEAX@Z 0000000180003fa0 f   MSVCRT:dll_dllmain.obj
 0001:000030b8       ?dllmain_crt_process_detach@@YAH_N@Z 00000001800040b8 f   MSVCRT:dll_dllmain.obj
 0001:0000313c       ?dllmain_dispatch@@YAHQEAUHINSTANCE__@@KQEAX@Z 000000018000413c f   MSVCRT:dll_dllmain.obj
 0001:00003b50       $$000000                   0000000180004b50     MSVCRT:guard_dispatch.obj
 0001:00003b70       $$000000                   0000000180004b70     MSVCRT:guard_xfg_dispatch.obj
 0001:00003b86       ?fin$0@?0??dllmain_crt_process_attach@@YAHQEAUHINSTANCE__@@QEAX@Z@4HA 0000000180004b86 f   MSVCRT:dll_dllmain.obj
 0001:00003b9d       ?fin$0@?0??dllmain_crt_process_detach@@YAH_N@Z@4HA 0000000180004b9d f   MSVCRT:dll_dllmain.obj
 0001:00003bb6       ?fin$1@?0??dllmain_crt_process_detach@@YAH_N@Z@4HA 0000000180004bb6 f   MSVCRT:dll_dllmain.obj
 0001:00003bca       ?filt$0@?0??dllmain_dispatch@@YAHQEAUHINSTANCE__@@KQEAX@Z@4HA 0000000180004bca f   MSVCRT:dll_dllmain.obj
 0001:00003c00       __scrt_is_nonwritable_in_current_image$filt$0 0000000180004c00 f   MSVCRT:utility.obj
 0002:000001e8       ?__scrt_initialize_tss_var@@3P6AHXZEA 00000001800051e8     MSVCRT:thread_safe_statics.obj
 0002:00000310       ?opcLengths@@3QBEB         0000000180005310     libgetlocal001.obj
 0002:00002368       GS_ExceptionPointers       0000000180007368     MSVCRT:gs_report.obj
 0002:00002a20       $unwind$fprintf            0000000180007a20     libgetlocal001.obj
 0002:00002a2c       $unwind$printf             0000000180007a2c     libgetlocal001.obj
 0002:00002a38       $unwind$?NewObject@JNIEnv_@@QEAAPEAV_jobject@@PEAV_jclass@@PEAU_jmethodID@@ZZ 0000000180007a38     libgetlocal001.obj
 0002:00002a38       $unwind$nsk_lcomplain      0000000180007a38     libgetlocal001.obj
 0002:00002a38       $unwind$nsk_ldisplay       0000000180007a38     libgetlocal001.obj
 0002:00002a40       $unwind$nsk_lvdisplay      0000000180007a40     libgetlocal001.obj
 0002:00002a40       $unwind$_RTC_Initialize    0000000180007a40     MSVCRT:initsect.obj
 0002:00002a40       $unwind$_RTC_Terminate     0000000180007a40     MSVCRT:initsect.obj
 0002:00002a40       $unwind$?__scrt_initialize_thread_safe_statics@@YAHXZ 0000000180007a40     MSVCRT:thread_safe_statics.obj
 0002:00002a4c       $unwind$nsk_lvcomplain     0000000180007a4c     libgetlocal001.obj
 0002:00002a64       $unwind$nsk_ltrace         0000000180007a64     libgetlocal001.obj
 0002:00002a64       $unwind$__report_gsfailure 0000000180007a64     MSVCRT:gs_report.obj
 0002:00002a6c       $unwind$Agent_Initialize   0000000180007a6c     libgetlocal001.obj
 0002:00002a6c       $unwind$nsk_lvtrace        0000000180007a6c     libgetlocal001.obj
 0002:00002a6c       $unwind$__raise_securityfailure 0000000180007a6c     MSVCRT:gs_report.obj
 0002:00002a6c       $unwind$__scrt_initialize_crt 0000000180007a6c     MSVCRT:utility.obj
 0002:00002a6c       $unwind$__scrt_initialize_onexit_tables 0000000180007a6c     MSVCRT:utility.obj
 0002:00002a6c       $unwind$__scrt_release_startup_lock 0000000180007a6c     MSVCRT:utility.obj
 0002:00002a6c       $unwind$__scrt_uninitialize_crt 0000000180007a6c     MSVCRT:utility.obj
 0002:00002a6c       $unwind$_onexit            0000000180007a6c     MSVCRT:utility.obj
 0002:00002a74       $unwind$nsk_lverify        0000000180007a74     libgetlocal001.obj
 0002:00002a84       $unwind$nsk_vprintf        0000000180007a84     libgetlocal001.obj
 0002:00002a94       $unwind$nsk_printf         0000000180007a94     libgetlocal001.obj
 0002:00002a9c       $unwind$?nsk_jni_lverify@@YAHHPEAUJNIEnv_@@HQEBDH1ZZ 0000000180007a9c     libgetlocal001.obj
 0002:00002ab0       $unwind$?nsk_jni_check_exception@@YAHPEAUJNIEnv_@@QEBDH@Z 0000000180007ab0     libgetlocal001.obj
 0002:00002acc       $unwind$Java_nsk_jvmti_unit_FollowReferences_FollowRefObjects_resetTags 0000000180007acc     libgetlocal001.obj
 0002:00002acc       $unwind$addRefToVerify     0000000180007acc     libgetlocal001.obj
 0002:00002acc       $unwind$nsk_jvmti_resetAgentData 0000000180007acc     libgetlocal001.obj
 0002:00002acc       $unwind$__scrt_initialize_default_local_stdio_options 0000000180007acc     MSVCRT:default_local_stdio_options.obj
 0002:00002acc       $unwind$?dllmain_crt_dispatch@@YAHQEAUHINSTANCE__@@KQEAX@Z 0000000180007acc     MSVCRT:dll_dllmain.obj
 0002:00002acc       $unwind$DllMain            0000000180007acc     MSVCRT:dll_dllmain_stub.obj
 0002:00002acc       $unwind$__GSHandlerCheck   0000000180007acc     MSVCRT:gshandler.obj
 0002:00002acc       $unwind$?__scrt_uninitialize_thread_safe_statics@@YAXXZ 0000000180007acc     MSVCRT:thread_safe_statics.obj
 0002:00002acc       $unwind$__scrt_acquire_startup_lock 0000000180007acc     MSVCRT:utility.obj
 0002:00002acc       $unwind$__scrt_dllmain_after_initialize_c 0000000180007acc     MSVCRT:utility.obj
 0002:00002acc       $unwind$__scrt_dllmain_before_initialize_c 0000000180007acc     MSVCRT:utility.obj
 0002:00002acc       $unwind$__scrt_dllmain_crt_thread_attach 0000000180007acc     MSVCRT:utility.obj
 0002:00002acc       $unwind$__scrt_dllmain_crt_thread_detach 0000000180007acc     MSVCRT:utility.obj
 0002:00002acc       $unwind$__scrt_dllmain_uninitialize_c 0000000180007acc     MSVCRT:utility.obj
 0002:00002acc       $unwind$__scrt_dllmain_uninitialize_critical 0000000180007acc     MSVCRT:utility.obj
 0002:00002acc       $unwind$atexit             0000000180007acc     MSVCRT:utility.obj
 0002:00002ad4       $unwind$nsk_jvmti_lverify  0000000180007ad4     libgetlocal001.obj
 0002:00002ae8       $unwind$exitOnError        0000000180007ae8     libgetlocal001.obj
 0002:00002af8       $unwind$Java_nsk_share_jvmti_ArgumentHandler_getAgentOptionsString 0000000180007af8     libgetlocal001.obj
 0002:00002b0c       $unwind$Java_nsk_jvmti_unit_FollowReferences_FollowRefObjects_getTag 0000000180007b0c     libgetlocal001.obj
 0002:00002b0c       $unwind$Java_nsk_share_jvmti_DebugeeClass_checkStatus 0000000180007b0c     libgetlocal001.obj
 0002:00002b0c       $unwind$agentThreadWrapper 0000000180007b0c     libgetlocal001.obj
 0002:00002b1c       $unwind$startAgentThreadWrapper 0000000180007b1c     libgetlocal001.obj
 0002:00002b38       $unwind$syncDebuggeeStatus 0000000180007b38     libgetlocal001.obj
 0002:00002b38       $unwind$__scrt_dllmain_exception_filter 0000000180007b38     MSVCRT:utility.obj
 0002:00002b4c       $unwind$Java_nsk_share_jvmti_DebugeeClass_resetAgentData 0000000180007b4c     libgetlocal001.obj
 0002:00002b54       $unwind$MA_checkStatus     0000000180007b54     libgetlocal001.obj
 0002:00002b68       $unwind$Java_nsk_jvmti_unit_FollowReferences_FollowRefObjects_setTag 0000000180007b68     libgetlocal001.obj
 0002:00002b80       $unwind$Java_nsk_jvmti_unit_FollowReferences_FollowRefObjects_addRefToVerify 0000000180007b80     libgetlocal001.obj
 0002:00002b9c       $unwind$check1             0000000180007b9c     libgetlocal001.obj
 0002:00002bbc       $unwind$check2             0000000180007bbc     libgetlocal001.obj
 0002:00002bd8       $unwind$check3             0000000180007bd8     libgetlocal001.obj
 0002:00002bf8       $unwind$check4             0000000180007bf8     libgetlocal001.obj
 0002:00002c14       $unwind$MethodExit         0000000180007c14     libgetlocal001.obj
 0002:00002c2c       $unwind$Breakpoint         0000000180007c2c     libgetlocal001.obj
 0002:00002c44       $unwind$Java_nsk_jvmti_GetLocalVariable_getlocal001_getMeth 0000000180007c44     libgetlocal001.obj
 0002:00002c44       $unwind$_DllMainCRTStartup 0000000180007c44     MSVCRT:dll_dllmain.obj
 0002:00002c54       $unwind$capture_previous_context 0000000180007c54     MSVCRT:gs_report.obj
 0002:00002c60       $unwind$__GSHandlerCheckCommon 0000000180007c60     MSVCRT:gshandler.obj
 0002:00002c68       $xdatasym                  0000000180007c68     MSVCRT:amdsecgs.obj
 0002:00002c6c       $unwind$?dllmain_crt_process_attach@@YAHQEAUHINSTANCE__@@QEAX@Z 0000000180007c6c     MSVCRT:dll_dllmain.obj
 0002:00002ca8       $unwind$?fin$0@?0??dllmain_crt_process_attach@@YAHQEAUHINSTANCE__@@QEAX@Z@4HA 0000000180007ca8     MSVCRT:dll_dllmain.obj
 0002:00002ca8       $unwind$?fin$0@?0??dllmain_crt_process_detach@@YAH_N@Z@4HA 0000000180007ca8     MSVCRT:dll_dllmain.obj
 0002:00002ca8       $unwind$?fin$1@?0??dllmain_crt_process_detach@@YAH_N@Z@4HA 0000000180007ca8     MSVCRT:dll_dllmain.obj
 0002:00002cb0       $unwind$?dllmain_crt_process_detach@@YAH_N@Z 0000000180007cb0     MSVCRT:dll_dllmain.obj
 0002:00002d04       $unwind$?dllmain_dispatch@@YAHQEAUHINSTANCE__@@KQEAX@Z 0000000180007d04     MSVCRT:dll_dllmain.obj
 0002:00002d2c       $unwind$?filt$0@?0??dllmain_dispatch@@YAHQEAUHINSTANCE__@@KQEAX@Z@4HA 0000000180007d2c     MSVCRT:dll_dllmain.obj
 0002:00002d34       $unwind$__scrt_is_nonwritable_in_current_image 0000000180007d34     MSVCRT:utility.obj
 0002:00002d54       $unwind$__scrt_is_nonwritable_in_current_image$filt$0 0000000180007d54     MSVCRT:utility.obj
 0002:00002d5c       $unwind$__scrt_fastfail    0000000180007d5c     MSVCRT:utility_desktop.obj
 0002:00002d6c       $unwind$__security_init_cookie 0000000180007d6c     MSVCRT:gs_support.obj
 0002:00002d78       $unwind$__isa_available_init 0000000180007d78     MSVCRT:cpu_disp.obj
 0002:00002d88       $xdatasym                  0000000180007d88     MSVCRT:guard_dispatch.obj
 0002:00002d90       $xdatasym                  0000000180007d90     MSVCRT:guard_xfg_dispatch.obj
 0002:00002da0       .edata                     0000000180007da0     getlocal001.exp
 0002:00002dc8       rgpv                       0000000180007dc8     getlocal001.exp
 0002:00002e08       rgszName                   0000000180007e08     getlocal001.exp
 0002:00002e48       rgwOrd                     0000000180007e48     getlocal001.exp
 0002:00002e68       szName                     0000000180007e68     getlocal001.exp
 0002:00002e78       $N00001                    0000000180007e78     getlocal001.exp
 0002:00002e87       $N00002                    0000000180007e87     getlocal001.exp
 0002:00002e94       $N00003                    0000000180007e94     getlocal001.exp
 0002:00002ec8       $N00004                    0000000180007ec8     getlocal001.exp
 0002:00002efb       $N00005                    0000000180007efb     getlocal001.exp
 0002:00002f40       $N00006                    0000000180007f40     getlocal001.exp
 0002:00002f7d       $N00007                    0000000180007f7d     getlocal001.exp
 0002:00002fc5       $N00008                    0000000180007fc5     getlocal001.exp
 0002:00003005       $N00009                    0000000180008005     getlocal001.exp
 0002:00003042       $N00010                    0000000180008042     getlocal001.exp
 0002:0000307d       $N00011                    000000018000807d     getlocal001.exp
 0002:000030ab       $N00012                    00000001800080ab     getlocal001.exp
 0002:000030dc       $N00013                    00000001800080dc     getlocal001.exp
 0002:0000310b       $N00014                    000000018000810b     getlocal001.exp
 0002:0000313a       $N00015                    000000018000813a     getlocal001.exp
 0002:0000316f       $N00016                    000000018000816f     getlocal001.exp
 0002:0000357a       .idata$6                   000000018000857a     kernel32:KERNEL32.dll
 0002:000035de       .idata$6                   00000001800085de     vcruntime:VCRUNTIME140.dll
 0002:0000374a       .idata$6                   000000018000874a     ucrt:api-ms-win-crt-runtime-l1-1-0.dll
 0002:0000376c       .idata$6                   000000018000876c     ucrt:api-ms-win-crt-stdio-l1-1-0.dll
 0002:0000378c       .idata$6                   000000018000878c     ucrt:api-ms-win-crt-string-l1-1-0.dll
 0003:00000000       ?codeAttributeName@@3PEBDEB 0000000180009000     libgetlocal001.obj
 0003:00000008       ?lineNumberAttributeName@@3PEBDEB 0000000180009008     libgetlocal001.obj
 0003:00000010       ?localVarAttributeName@@3PEBDEB 0000000180009010     libgetlocal001.obj
 0003:00000018       ?localVarTypeAttributeName@@3PEBDEB 0000000180009018     libgetlocal001.obj
 0003:00000020       ?stackMapAttributeName@@3PEBDEB 0000000180009020     libgetlocal001.obj
 0003:00000028       ?callBytes@@3PAEA          0000000180009028     libgetlocal001.obj
 0003:0000002c       ?allocBytes@@3PAEA         000000018000902c     libgetlocal001.obj
 0003:0001aad4       redefineAttempted          0000000180023ad4     libgetlocal001.obj
 0003:0001aad8       nsk_context                0000000180023ad8     libgetlocal001.obj
 0003:0001aae4       redefineSucceed            0000000180023ae4     libgetlocal001.obj
 0003:0001aae8       agentFailed                0000000180023ae8     libgetlocal001.obj
 0003:0001aaec       currentAgentStatus         0000000180023aec     libgetlocal001.obj
 0003:0001aaf0       context                    0000000180023af0     libgetlocal001.obj
 0003:0001aba8       agentThread                0000000180023ba8     libgetlocal001.obj
 0003:0001abb0       agentThreadProc            0000000180023bb0     libgetlocal001.obj
 0003:0001abb8       agentThreadArg             0000000180023bb8     libgetlocal001.obj
 0003:0001abc0       agent_data                 0000000180023bc0     libgetlocal001.obj
 0003:0001abd0       jvmti_env                  0000000180023bd0     libgetlocal001.obj
 0003:0001abd8       jvm                        0000000180023bd8     libgetlocal001.obj
 0003:0001abe0       jni_env                    0000000180023be0     libgetlocal001.obj
 0003:0001abe8       checkStatus_func           0000000180023be8     libgetlocal001.obj
 0003:0001abf0       ?codeAttributeIndex@@3GA   0000000180023bf0     libgetlocal001.obj
 0003:0001abf2       printdump                  0000000180023bf2     libgetlocal001.obj
 0003:0001abf4       ?lineNumberAttributeIndex@@3GA 0000000180023bf4     libgetlocal001.obj
 0003:0001abf8       ?localVarAttributeIndex@@3GA 0000000180023bf8     libgetlocal001.obj
 0003:0001abfc       ?localVarTypeAttributeIndex@@3GA 0000000180023bfc     libgetlocal001.obj
 0003:0001ac00       ?stackMapAttributeIndex@@3GA 0000000180023c00     libgetlocal001.obj
 0003:0001ac04       ?stackFrameOffset@@3GA     0000000180023c04     libgetlocal001.obj
 0003:0001ac08       ?mode@@3HA                 0000000180023c08     libgetlocal001.obj
 0003:0001ac0c       ?constantPoolSize@@3GA     0000000180023c0c     libgetlocal001.obj
 0003:0001ac10       ?orig@@3PEBEEB             0000000180023c10     libgetlocal001.obj
 0003:0001ac18       ?gen@@3PEAEEA              0000000180023c18     libgetlocal001.obj
 0003:0001ac20       ?inputPos@@3PEAEEA         0000000180023c20     libgetlocal001.obj
 0003:0001ac28       ?endPos@@3PEBEEB           0000000180023c28     libgetlocal001.obj
 0003:0001ac30       ?genPos@@3PEAEEA           0000000180023c30     libgetlocal001.obj
 0003:0001ac38       ?markPos@@3PEAEEA          0000000180023c38     libgetlocal001.obj
 0003:0001ac40       ?constantPool@@3PEAPEADEA  0000000180023c40     libgetlocal001.obj
 0003:0001ac48       ?constantPoolCount@@3GA    0000000180023c48     libgetlocal001.obj
 0003:0001ac4c       ?zeroBytes@@3PAEA          0000000180023c4c     libgetlocal001.obj
 0003:0001ac50       ?codeLength@@3IA           0000000180023c50     libgetlocal001.obj
 0003:0001ac54       result                     0000000180023c54     libgetlocal001.obj
 0003:0001ac58       ?map@@3PEAIEA              0000000180023c58     libgetlocal001.obj
 0003:0001ac60       ?widening@@3PEACEA         0000000180023c60     libgetlocal001.obj
 0003:0001ac68       jvmti                      0000000180023c68     libgetlocal001.obj
 0003:0001ac70       caps                       0000000180023c70     libgetlocal001.obj
 0003:0001ac80       callbacks                  0000000180023c80     libgetlocal001.obj
 0003:0001adb8       mid1                       0000000180023db8     libgetlocal001.obj
 0003:0001adc0       mid2                       0000000180023dc0     libgetlocal001.obj
 0003:0001adc8       mid3                       0000000180023dc8     libgetlocal001.obj
 0003:0001add0       mid4                       0000000180023dd0     libgetlocal001.obj
 0003:0001add8       fval                       0000000180023dd8     libgetlocal001.obj
 0003:0001ade0       dval                       0000000180023de0     libgetlocal001.obj
 0003:0001adf0       GS_ExceptionRecord         0000000180023df0     MSVCRT:gs_report.obj
 0003:0001ae90       GS_ContextRecord           0000000180023e90     MSVCRT:gs_report.obj
 0003:0001b360       ?g_tss_cv@@3U_RTL_CONDITION_VARIABLE@@A 0000000180024360     MSVCRT:thread_safe_statics.obj
 0003:0001b368       ?g_tss_event@@3PEAXEA      0000000180024368     MSVCRT:thread_safe_statics.obj
 0003:0001b370       ?g_tss_mutex@@3U_RTL_CRITICAL_SECTION@@A 0000000180024370     MSVCRT:thread_safe_statics.obj
 0003:0001b398       ?g_sleep_condition_variable_cs@@3P6AHPEAU_RTL_CONDITION_VARIABLE@@PEAU_RTL_CRITICAL_SECTION@@K@ZEA 0000000180024398     MSVCRT:thread_safe_statics.obj
 0003:0001b3a0       ?g_wake_all_condition_variable@@3P6AXPEAU_RTL_CONDITION_VARIABLE@@@ZEA 00000001800243a0     MSVCRT:thread_safe_statics.obj
 0003:0001b3ac       ?__proc_attached@@3HA      00000001800243ac     MSVCRT:dll_dllmain.obj
 0003:0001b3c0       ?is_initialized_as_dll@@3_NA 00000001800243c0     MSVCRT:utility.obj
 0003:0001b3c1       ?module_local_atexit_table_initialized@@3_NA 00000001800243c1     MSVCRT:utility.obj
 0003:0001b3c8       ?module_local_atexit_table@@3U_onexit_table_t@@A 00000001800243c8     MSVCRT:utility.obj
 0003:0001b3e0       ?module_local_at_quick_exit_table@@3U_onexit_table_t@@A 00000001800243e0     MSVCRT:utility.obj
